:10000000E84300208D8C000001CA011001CA0110D4
:1000100001CA011001CA011001CA011001CA011070
:1000200001CA011001CA011001CA011001CA011060
:0C00300001CA011001CA01103FCA0110F2
:10003C00F3010100012002A80700201712000100A3
:10004C0002C80600205200015200011200010002F9
:04005C000800000098
:100100003C0000000000000000000000340100007E
:1001100000000000000000000100000000000000DE
:1001200000000000000000000000000001000000CE
:0C013000000000000800000000000000BB
:10013C003400000000000000000000006801000016
:10014C0000000000000000000100000000000000A2
:10015C00010000000000000000000000080000008A
:04016C00000000008F
:1001700030000000000000000000000098010000B6
:10018000040000000000000001000000FFFFFFFF6E
:10019000FF00000001000000080000000000000057
:1001A0002C0000000000000000000000C40100005E
:1001B000040000000000000001000000FFFFFFFF3E
:0C01C000FFFFFFFF08000000000000002F
:1001CC0034050000E401000099A1011095A701106D
:1001DC00A5C2011009B2011045B8011000000000C1
:0801EC00000000002E000000DD
:1001F40028000000000000000000000014020000BD
:100204000000000000000000FFFFFFFF00000000EE
:080214000800000000000000DA
:10021C00300500003002000069C201106DC10110F0
:10022C001FC2011095BA0110000000000000000070
:04023C00300000008E
:10024000300500005402000075C20110A9B601106B
:100250009DBF011049B60110000000000000000021
:040260003100000069
:1002640024000000000000000000000080020000E4
:100274000000000000000000000000000800000072
:040284000000000076
:10028800240000000000000000000000A40200009C
:10029800000000000000000000000000080000004E
:0402A8000000000052
:1002AC00240000000000000000000000C802000054
:1002BC000000000001000000000000000800000029
:0402CC00000000002E
:1002D00000000000300900200400000000000000C1
:1002E000000000002000000070010000300000004D
:1002F0001C0200003809002004000000000000007B
:10030000000000000C000000300400001800000095
:10031000400200004009002004000000000000002E
:100320000000000024000000480400001800000045
:100330000000000048090020040000000000000048
:100340000000000010000000A00100002C000000D0
:10035000CC01000050090020040000000000000053
:1003600000000000200000006402000024000000E3
:10037000FFFFFFFF580900200400000000000000FC
:100380000000000028000000880200002400000097
:10039000FFFFFFFF680900200400000000000000CC
:1003A00000000000580000003C0100003400000084
:1003B000FFFFFFFF700900200400000000000000A4
:1003C00000000000100000006004000018000000A1
:1003D000FFFFFFFF7809002004000000000000007C
:1003E000000000001C000000AC020000240000001F
:1003F000FFFFFFFF80090020040000000000000054
:100400000000000038000000F40100002800000097
:10041000FFFFFFFF8809002004000000000000002B
:100420000000000054000000000100003C0000003B
:100430001800000000000000000000004004000060
:080440000800000000000000AC
:100448001800000000000000000000005804000030
:08045800080000000000000094
:100460001800000000000000000000007004000000
:0804700008000000000000007C
:0804780001000000888D000066
:040484000100000073
:0404880000000C0064
:04048C0000000D005F
:040490003200000036
:040494000200000062
:0404980048070020F1
:04049C00000200005A
:0404A0000000000058
:0404A40001CA011078
:0404A8000000000050
:0404AC00000000004C
:0404B0000800000040
:0404B4000000200024
:0404B8001007002009
:0404BC00010000003B
:0404C000CC08002044
:0404C400080000002C
:0404C8000000000030
:0404CC00000000002C
:0404D0000000000028
:0404D4000000000024
:0404D8000000000020
:0404DC00010000001B
:0404E0007807002079
:0404E400060000000E
:0404E800010000000F
:0404EC007C0600206A
:0404F0000000000008
:0404F4000000000004
:0404F80000020000FE
:0404FC0000000000FC
:020502002A00CD
:020504000100F4
:020506002500CE
:020508003000C1
:02050A003100BE
:02050C002E00BF
:02050E000100EA
:0105100001E9
:0805140004000000B88C000097
:08051C000000000000000000D7
:0405240000000100D2
:0405280000000300CC
:04052C0087C401106F
:04053000380500008A
:040534003805000086
:0405380000000000BF
:04053C00800000003B
:040540008000000037
:0405440000000000B3
:04054800CC080020BB
:04054C00131E00007A
:040550002000000087
:04055400A48C000073
:0405580018F701008F
:04055C000DC30110BA
:040560008D150000F5
:040564008F150000EF
:0405680099C801101D
:04056C009BC8011017
:040570000000000087
:04057400222300003E
:04057800C0F50100C9
:04057C00D8F50100AD
:04058000A8F50100D9
:0205840008006D
:0205860009006A
:02058800010070
:02058A0000006F
:01058C00016D
:040590000000000067
:040594000000000063
:04059800000000005F
:04059C00000000005B
:0405A000291400001A
:0405A40089140000B6
:0405A8000913000033
:0405AC00B314000084
:0405B00071130000C3
:0405B4002713000009
:0405B800B11300007B
:0405BC00F514000032
:0405C000911D000089
:0405C400931F000081
:0405C800971F000079
:0405CC000800000023
:0405D0002400000003
:0405D400180000000B
:0405D80028000000F7
:0405DC0020000000FB
:0405E0003C000000DB
:0405E4000C00000007
:0405E80034000000DB
:1005EC00DFF800F0F5C00110DFF800F049BA011097
:1005FC00DFF800F0E5C10110DFF800F025C20110B2
:10060C00DFF800F0C1C20110DFF800F0E3BF011009
:10061C00DFF800F013C10110DFF800F0B5C10110D4
:10062C00DFF800F0D5C20110DFF800F0F5B80110CA
:10063C00DFF800F0D5C00110DFF800F0F1C50110B3
:10064C00DFF800F095C00110DFF800F00DA80110E4
:10065C00DFF800F0BDBE0110DFF800F021C1011081
:10066C00DFF800F0A5B90110DFF800F021BA011095
:10067C00DFF800F0BDC20110DFF800F015B6011074
:10068C00DFF800F019A70110DFF800F02DBF011002
:10069C00DFF800F0E1B50110DFF800F0D9C201106D
:1006AC00DFF87C02007D704738B5DFF87C02DFF89C
:1006BC0074520068EFF3118480F31188A86800214C
:1006CC00FFF7BEFF6969081AA969814238BF00208B
:1006DC0084F3118832BD00002DE9F041DFF84802A7
:1006EC00DFF840420768EFF3118887F31188A068A0
:1006FC000121FFF7A5FF0121A1830021E183656999
:10070C0021682268461B801A691A884204D200208C
:10071C00A08388F311882AE088F31188002005E073
:10072C004519361A29460120FFF78EFF8642F7D26B
:10073C00EFF3118887F31188E18B012903D1294646
:10074C000020FFF781FFA16910F1010F08BF0846D7
:10075C0003D0801B814238BF08464119FFF778FF50
:10076C00012020840020A083256088F31188BDE837
:10077C00F081808A70470021DFF8B0210160126897
:10078C001044FFF751BF000038B500F0D3F8EFF379
:10079C00118580F31188207C022808D12046FFF7B0
:1007AC005BFF002020742946A068FFF759FF85F3F2
:1007BC00118831BD03681A4003680B408B4208BF97
:1007CC000A4312B101689143016010467047000062
:1007DC002DE9F0431F4617F1010F18BF002F91B000
:1007EC0004460D4616460AD06B463A46DFF84011D1
:1007FC0008A8FFF739FF08A80390022002E00020A8
:10080C00039003208DF8100006950796FFF7F0FE75
:10081C0002903246DFF81001D0F80080EFF3118916
:10082C0088F3118829462046FFF7C4FF050007D03E
:10083C00039808B1FFF71CFF89F31188284633E0B1
:10084C001FB989F3118800202EE0FFF7C9FE054679
:10085C000299DFF8D800C1F818D069460068204426
:10086C00FFF7DAFE0298FFF707FF9DF81000022849
:10087C0004BF0398FFF704FF89F311882846FFF79C
:10088C00B3FEEFF3118488F31188039818B1FFF7C6
:10089C00EFFE0020039000200299886184F31188F8
:1008AC009DF8100000B1059811B0BDE8F083000070
:1008BC00F8B50446DFF874000068261800F03BF821
:1008CC00EFF3118580F311882068084320603046CF
:1008DC00FFF79EFE10B185F31188F1BDFFF780FE86
:1008EC0007463046FFF79CFE0646F269B169204682
:1008FC00FFF760FF706160B13046FFF7ADFE01207D
:10090C003074F06808B1FFF777FEB0682946FFF73E
:10091C00A7FE85F311883846BDE8F240FFF764BEA8
:10092C00A4010020780100207C8D0000848D000043
:10093C009507000004460148006870477C8D000054
:10094C00DFF80410096870477C8D000000F01ABEB7
:10095C0080B5002301223421DFF8F00901F0D0F832
:10096C0000B10120C0B202BDDFF8C41A0A68002829
:10097C0012BF42F0010050084000086070470000B0
:10098C007047FEE710B582B0042001F0F1F80228A0
:10099C0018BF03280DD1032000901C234FF04052A8
:1009AC000021DFF8A80901F088F8BDE81640042002
:1009BC006AE0DFF89C19DFF89C0A09684418DFF834
:1009CC009419DFF8940A0968B0FBF1F12046FFF79F
:1009DC0017FE2046BDE81640FFF716BE80B5DFF8BF
:1009EC0078090078DFF8740901688908890041F0FA
:1009FC000101016001F0C9F801F053F9DFF8601949
:100A0C00002008600220DFF894190968C96888473B
:100A1C00DFF85C0A016849084900016000F01BFA24
:100A2C00042000F013F900F0B6BC0000DFF82C1A1B
:100A3C00085C70470022012904D1012807D1DFF896
:100A4C00600903E0012802D1DFF82C0A0268104685
:100A5C007047DFF8000A00797047000001F0AAB86F
:100A6C0010B5DFF83C160968EFF3118481F3118897
:100A7C00DFF8E019C9880120012908BFFFF768FFDA
:100A8C0084F3118810BD000030B5DFF81416DFF8C0
:100A9C0088390A68EFF3118182F31188B0FA80F279
:100AAC00C2F11F029A5CB0FA80F4C4F11F04551E07
:100ABC001D5505D1DFF89C29136823EA000010604E
:100ACC0081F3118830BD00002DE9F041FFF738FFAC
:100ADC00EFF3118481F31188DFF880190A5C531E3F
:100AEC000B5444D1DFF87819DFF8788901EB8005D5
:100AFC002E786F88300618D5D8F80010096A384659
:100B0C008847D8F80010896A38468847D8F800100A
:100B1C00096B38468847DFF8501901200860DFF868
:100B2C004C0900688007FAD514E0700606D5DFF88A
:100B3C00AC1951F82710002088470BE0D8F80010AA
:100B4C00896938468847D8F80010496B3846884779
:100B5C000228F8D106F03F003F2818BFFFF7B4FF7A
:100B6C00687800F03F003F2818BFFFF7ADFF84F313
:100B7C001188BDE8F08110B508B1140001D1032033
:100B8C0010BD8160C26003610146DFF8E828DFF820
:100B9C00500912681044FFF777FD002010BD0000CB
:100BAC00F8B50446DFF8F804DFF8B0180068EFF386
:100BBC00118580F311880A5D531C0B55002A3ED118
:100BCC00DFF89C1801EB8407387800F03F003F28D1
:100BDC0018BFFFF7E5FF787800F03F003F2818BFFB
:100BEC00FFF7DEFF7E883878DFF87878010613D5BA
:100BFC003968C969304688473968496A3046884738
:100C0C003968C96A3046884700F038F8DFF85C0864
:100C1C0000688007FAD512E0400606D5DFF8BC184C
:100C2C0051F826100120884709E039684969304697
:100C3C0088473968496B304688470128F9D185F3D4
:100C4C0011882046BDE8F24001F08AB9DFF8501453
:100C5C000A68EFF3118182F31188DFF8F827136823
:100C6C0003431360B0FA80F0C0F11F00DFF8A8272F
:100C7C00135C5B1C135481F311887047DFF8E81781
:100C8C0001200860704700002DE9F04F4FF000087C
:100C9C000021012883B0C1468A4618BF022412D114
:100CAC00DFF8FC03DFF838780268EFF3118082F389
:100CBC0011883A79012A06BF02223A71012180F388
:100CCC00118809B10624BDE0FFF78AFC00900120D1
:100CDC0000F0E6F8044610B101203871AFE0FFF7E0
:100CEC00A7FCDFF828180190C1F80090012000F053
:100CFC003FFF012804D1002001F012F94FF0010848
:100D0C00DFF8E047DFF854572168896800208847EE
:100D1C0000F0A1F8687C08B14FF00109287C08B1FB
:100D2C0049F00209E87B08B149F00409E87ADFF8D8
:100D3C00306718B1A16AF08D096B8847A87A18B191
:100D4C00A16A708D096B8847FFF798FF49F0200066
:100D5C00A16A896988470120FFF706FE3878C00729
:100D6C0048BF4FF0010A12D4DFF8980701F03EF9A2
:100D7C008346BBF1040FF7D000F067F880088000C1
:100D8C0008600321A26CDFF87C07526890470020B2
:100D9C0001F034F900F05FF8A06A806B8047BAF17B
:100DAC00000F0AD1A26CDFF85C07526859469047D5
:100DBC0000F04BF840F003000860012021688968BE
:100DCC008847DFF8440700688006FAD5B8F1000FB1
:100DDC001CBF012001F0A4F8A16A49694846884764
:100DEC00A16A496B484688470128F9D1E87A18B1BD
:100DFC00A16AF08DC96A8847A87A18B1A16A708D6A
:100E0C00C96A8847FFF73AFF0020FFF7ADFD0320C2
:100E1C003871042000F044F8DFF8F0160120086067
:100E2C0000F019F801F0F8F9082000F039F8044640
:100E3C00012038710198FFF72BFC01F078F900982C
:100E4C00FFF7D2FB2046BDE8FE8FDFF8D006DFF8B7
:100E5C00CC1600687047DFF8A806006870470000E1
:100E6C0038B58F48DFF878560068EFF3118480F3BB
:100E7C001188E888012803D100F0F0FE0020E880FA
:100E8C0084F3118831BD000010B5FFF759FDEFF365
:100E9C00118481F31188FFF7DFFB84F3118810BDF7
:100EAC0038B500F02AF80844FFF7B2FB002540B92A
:100EBC00204600F008F820B1DFF86806006880478B
:100ECC000225284632BD70B500F017F845182846A3
:100EDC00FFF7A6FB0646B068204206D03169F268DF
:100EEC0020469047C0B2012806D03046FFF7D4FB0D
:100EFC000646AE42EFD1002070BDDFF878150968C8
:100F0C000446DFF8DC05704730BF704770B501F060
:100F1C007FF9DFF840552E6806F00C000C284BD0FA
:100F2C00700727D4FFF7C0FB044600210120FFF710
:100F3C0081FDA0421ED2DFF8C00300680544DFF833
:100F4C0014040668DFF8D8050068B0FBF6F0211A27
:100F5C002846FFF755FB2846FFF756FB4FF47A70EF
:100F6C00B0FBF6F200210120FFF78EFE2846FFF7BA
:100F7C0043FB23E030071FD4DFF8F404DFF8E4442C
:100F8C00DFF87C55F10601685ABF4908490041F069
:100F9C0001010160DFF88405016841F00301016083
:100FAC00202021688969884728682068806B8047E1
:100FBC0001202860286801E0FFF7A6FF01F02CF95A
:100FCC00BDE8704001F0DEB810B50C1801F020F946
:100FDC00401E8041C00FDFF860150A68002AFCD063
:100FEC00246801220A6008B101F016F9204610BDF0
:100FFC0080B50420FFF72AFE0820FFF727FE0E20FD
:10100C00FFF7CEFDDFF82005DFF820150068C0F3F0
:10101C00815003280CBF012000200880DFF8100548
:10102C0002680AB1012002BDDFF8103540221A60B7
:10103C000122C2610020486002BD10B5DFF85C13CC
:10104C00DFF8F04482B009680968202088470F2037
:10105C002060072341F61D5060604FF4C0720220DF
:10106C00009000F0C9F8DFF8D80401210160016894
:10107C008907FCD501212161DFF8B04421880129C1
:10108C0007D1002101610220202100F091F80120FC
:10109C0004E00121002000F08BF80220606013BDF9
:1010AC007C8D00002DE9F041DFF89804DFF87C44DA
:1010BC0082B0016842688A4342600161606800281E
:1010CC0004BFBDE8F341FFF7B8BF0128DFF878147F
:1010DC001AD10220606008684BF2F5214843618800
:1010EC00000A11B10021618006E0DFF86014096884
:1010FC0021F07F4108184008DFF854140860000CF8
:10110C004860012088600CE002280FD10868B0F517
:10111C00C06F02D10020606045E00321616000F0E7
:10112C006FF80121BDE8FC41002041E003283DD1CE
:10113C00002060600868A0F5C065A06800F0B2F8F7
:10114C000646284600F0AEF886422CDAA6692846F8
:10115C0000F0ACF88019A061E56860697B4E8542AF
:10116C000ED0A769A7F1100000F09CF8804620690A
:10117C00103800F097F8804502DABFB200970BE008
:10118C00ADB2009508234FF47F423021304600F079
:10119C0094FC206980B2009012234FF4F8020421D1
:1011AC00304600F08AFCBDE8F3418AE0BDE8F381EB
:1011BC0070B50D46DFF89C4382B0032121600021FD
:1011CC00DFF89463316031688907FCD480B20090F9
:1011DC000523602200F010F8012030603068800791
:1011EC00FCD5A561002020600821DFF85003C16008
:1011FC0001600120206073BD0021544800F05DBCEB
:10120C0070B50646514C82B030212046FFF7DCFE0B
:10121C00DFF81853C0F30720E86004212046FFF7DD
:10122C00D3FEC0F384402861A6F5C060A8602E6987
:10123C0000F03CF88019A861A969E868022909DA6C
:10124C00401E6FF03F039842B8BF184610310BD5C3
:10125C00002109E01E2908DB401C4028A8BF3F20C4
:10126C0010392029A8BF1F21A9616861082380B209
:10127C0000904FF47F42302100F011F801200090D3
:10128C0011234FF4003200F009F8A86980B20090E5
:10129C0012234FF4F80200F001F873BD042120462C
:1012AC0000F00BBC002848BF4042704700284CBFE0
:1012BC006FF00101022101EB4000032190FBF1F0E2
:1012CC00704780B5DFF8780200210160016889075A
:1012DC00FCD40021016041600120DFF85412086049
:1012EC000E20FFF7F1FB0820FFF7CEFBBDE8024014
:1012FC000420FFF7C9BB0000608D000010B5044648
:10130C000020D4E90A2347F6906100F08DFF0123F9
:10131C00994228BF4FF0FF3010BD10B50C4600F0BD
:10132C00FBFF011D201AB0F1004F05D8081BB0F1CE
:10133C00004F38BF8C4200D20C46DFF820221268D6
:10134C00526A2146BDE810400120104700A00C4015
:10135C00648D0000808D0000173F00200440034086
:10136C00401009402DE9F04180460A46D8E90A01AF
:10137C00D8E90C45A0FB026701FB0277A6196F4167
:10138C00340C002244EA07414046FFF7C6FFC8E987
:10139C000E67BDE8F0814FF0FF3002BDA0010010D8
:1013AC00708D0000F8B50546DFF8B801DFF8B861BC
:1013BC000068DFF8B871EFF3118480F3118830689E
:1013CC0040F0800030600120B96849688847F96AAC
:1013DC00096A142088472869BA68526AB0F5802FC8
:1013EC0034BF0421010C012090473A681268232174
:1013FC0000209047B968C96901208847306820F4FB
:10140C00E02040F480303060306840F00100306003
:10141C0084F31188F1BD0000CC3E0020DFF85401AC
:10142C0003684068002200211018594170470000E1
:10143C000C200840DFF82411DFF8240110B50968EE
:10144C0044684968012088476069A169BDE810407B
:10145C0008470000B8050020A0860100383E002097
:10146C00F0F50100B8010010282008602820084081
:10147C008C210840688D0000748D0000F8B504467E
:10148C000D46FFF7CBFFD4E90A6732463B4600F026
:10149C00CBFE3DB1A6FB002306FB013307FB00335B
:1014AC00C4E90C23F2BD38B5DFF8BC40DFF8C050FE
:1014BC002068400840002060206840F080002060D8
:1014CC000120E062E06A2968496801208847696A5E
:1014DC00096A14208847E06A31BD00001409002015
:1014EC00B80500209001001080B500F004F8000C45
:1014FC0040EA014002BDDFF8800000688EE7000082
:10150C002C20094000400340141009400C400940B5
:10151C0009B9DFF86810FFF78FB8000024220840E3
:10152C00788D00006C8D0000B43F005050080020F6
:10153C0004800C400C400C4000800C402C500C40A3
:10154C0034600C4028500C4008400C4010200940DE
:10155C003C600C4000400C4038600C408C0100108A
:10156C00E40100207C8D0000002009408401001063
:10157C008C01001008200940EC010020A0010000A3
:10158C00FEE7704710B5DFF86404046814F1010F2E
:10159C0008BF002400F034FFDFF85414002008606A
:1015AC000120DFF850140860DFF84C140860DFF8F5
:1015BC004C04006828B1DFF848040068204600F0AD
:1015CC0023F8DFF84004DFF840240168890889001B
:1015DC0041F0005141F005010160DFF83004016871
:1015EC006FF31B4111430160DFF824040168C1F360
:1015FC000131012907D10168DFF81824114041F4A9
:10160C0000320260016010BD2DE9F84F0446DFF88E
:10161C00081401200860DFF8040401680029FCD0DC
:10162C00DFF8FC53DFF8FC83C0202860D8F80CA04E
:10163C00D8F80810DFF8F00389075DBFD8F804105C
:10164C00090C41F0F00172210170DFF8E013096818
:10165C00D8F80C20C1F304611629A8BF203901EB7E
:10166C002271491C6FF009029142B8BF114601F07A
:10167C001F0141F4F8510183CAF3C061DFF8B003D4
:10168C0081F001010160CAF3806181F00101816088
:10169C0014B9DFF8A0732DE0DFF89C030068C0F3E9
:1016AC0083615FEA8A32C0F38F2021D44FEA0A4269
:1016BC0012160AD54FF6FF73400804D11846490894
:1016CC0004BF01210120521CF6D4012A10DB40007A
:1016DC0040F00100B0F5803F21BF0120490041F0EE
:1016EC000101102924BF0F214FF6FF70521EECE7A9
:1016FC0040EA014700F08CFD401E8041C00FCF4EE8
:10170C0031680029FCD0DFF83893C9F8107001213A
:10171C00316008B100F080FD0CB9D82008E0C64A51
:10172C0010681168C0F3870001F0030140EA012042
:10173C00009040F2FF3700233A462C21C14800F0BC
:10174C00BCF91CB1BC48C06A8704BF0C00F060FD3A
:10175C00401E8041C00F31680029FCD0C9F81470BC
:10176C000121316008B100F057FD002C0FBFB64FBE
:10177C00B148406A20F0033700F04AFD401E80411A
:10178C00C00F31680029FCD0C9F80C700121316000
:10179C0008B100F041FD0CB9AC4F04E0A648AC49CF
:1017AC00006A01EA000700F033FD401E8041C00FC3
:1017BC0031680029FCD0C9F808700121316008B1EA
:1017CC0000F02AFD0CB9A34F20E09B48806AD8F8A2
:1017DC000830DB07C0F30352C0F303410BD4D8F835
:1017EC0004301F0502EB27721B0482F3040201EB89
:1017FC00237181F30401090441EA025182B242EAE5
:10180C000107222C24BF00F08040074300F000FDAC
:10181C00401E8041C00F31680029FCD0C9F804700B
:10182C000121316008B100F0F7FC2220222C824FFC
:10183C0006D3F86B000F00F00100400040F02000D0
:10184C00854908721120222C05D3F86B400F00F04B
:10185C00010040F01000202C08724FF0000B07D351
:10186C00B86CC10C01F44071C0F3845040EA010B18
:10187C0000F0CEFC401E8041C00F31680029FCD026
:10188C00C9F820B00121316008B100F0C5FC60201E
:10189C00202C06D3B86C000D00F00300400040F083
:1018AC0060006D49C8728020222C06D3F86BC00EE4
:1018BC0000F00100C00040F080000870222C4FF4B2
:1018CC007C4006D3F86B400D00F03F00800040F4E4
:1018DC007C406249DFF888B10880202C0AD3B86CB0
:1018EC000203810A02F47C1242EA815100F00F00DB
:1018FC0041EA003B00F08CFC401E8041C00F316877
:10190C000029FCD0C9F800B00121316008B100F009
:10191C0083FC544844210170882181700CB930211A
:10192C0005E0F96BC90C01F0030141F03001C17005
:10193C004FEA9A5010F0030003D002283CD012D387
:10194C003CE00121042000F0F1F843F2BD70E863A3
:10195C008620286401206864434801680029FCD073
:10196C00002068642EE0012000F002F904462146B4
:10197C00042000F0DBF8042000F0FAF8A042FAD1C1
:10198C00D8F800301802000A81B2E963000C286410
:10199C0001206864344801680029FCD00020686488
:1019AC004FF06022180E314B1B681B6807219847BB
:1019BC004FF48060C9F83800032100E002210420B4
:1019CC0000F0B4F8F8692A4900F03F00087047F6B7
:1019DC001800284908801049274800680020286012
:1019EC000860012025490860BDE8F18F1C130050E8
:1019FC00840460425C600C4008220443800128434C
:101A0C0000012043044003400000390148200340FA
:101A1C0004000940FFFFFCFC101009409402224313
:101A2C0000600C40A83F005056620840B8120050AD
:101A3C0000002043FF0F0F005013005000800C409B
:101A4C0008A00C4000A00C40000088688A76680052
:101A5C00FFFFFC00273F710041A10C40DCA10C40B2
:101A6C0000803F4005A10C4084088C43B401001059
:101A7C000BB00C4070B00C402C2009409404604218
:101A8C0038B504460D4600F0C3FB401E8041C00F24
:101A9C001A490A68002AFCD0012D02D0022D02D06E
:101AAC0003E0247802E0248800E0246801220A6024
:101ABC0008B100F0B1FB204632BD38B500EB410057
:101ACC00102B00F5007402D3103B241D120C04984B
:101ADC00984040EA024500F09BFB401E8041C00F3D
:101AEC0006490A68002AFCD0256001220A600028F9
:101AFC001CBFBDE8314000F08FBB31BD00800C40F5
:101B0C0038B51D460818102D144602D3103D801C04
:101B1C00240C0221FFF7B4FF04EA000188B2E8406C
:101B2C0032BD0268531C03601170704738B504460F
:101B3C00E0070D4607D5A8B2009000230122002132
:101B4C006B48FFF7BAFFA00707D5A8B20090012396
:101B5C00022200216648FFF7B0FF600707D5ADB23F
:101B6C00009502230C2200216148FFF7A6FF31BD2E
:101B7C000146042907BF1D234FF0C0421C234FF020
:101B8C0080525B483421FFF7BBBF10B5594C21681C
:101B9C00896801208847584801688906FCD5216965
:101BAC0009684020884721698968402088471128A6
:101BBC00F9D110BD70B5054600F0AEFB4F4C616815
:101BCC00401A4FF47A714843060C00F023FC21694B
:101BDC00401A48BF4042711940F6B932914207D2BF
:101BEC00062805DAA068E168814201D3226852B95F
:101BFC0043494A68D2074FF4FA6016D40868C0B259
:101C0C007D21484308E0081A3E494843000C00EB8C
:101C1C009000904238BF1046C82801D2C82070BD31
:101C2C00B0F57A6F88BF4FF47A6070BD10B582B092
:101C3C000120009000232E4C012219462046FFF76C
:101C4C003CFF012000900346022200212046FFF7B2
:101C5C0034FF00F061FB2949886013BD80B5012079
:101C6C00FFF786FF01281AD00023012234212048D7
:101C7C00FFF746FFA0B124480068804700F04CFBFA
:101C8C001E498B680A68C860A2EB9202C01A1D4BF1
:101C9C005843000C0860904238BF10460860012081
:101CAC0002BD10B582B0002000900146104C0023FC
:101CBC0001222046FFF701FF00200090014601237E
:101CCC0002222046FFF7F9FE1C234FF080523421EC
:101CDC002046FFF715FF10B10B4800688047074CF2
:101CEC0000F01AFB606000F095FB206113BD000052
:101CFC0000A00C4090010010141009404C3E002034
:101D0C00AC3F005040420F0080000010DFF800F0A4
:101D1C0049C10110DFF800F019C20110DFF800F022
:101D2C0095B70110DFF800F00DC30110DFF800F0DB
:101D3C0081C60110DFF800F08DC20110DFF800F051
:101D4C003DC20110DFF800F009C30110DFF800F00C
:101D5C0045C00110DFF800F0D1C70110DFF800F02A
:101D6C0067BE0110DFF800F021B30110DFF800F0BE
:101D7C0011C80110DFF800F021C80110DFF800F0E5
:101D8C0039C601100C2811D0192814D01D2817D0D1
:101D9C0020281AD021281DD0252820D02A2823D04D
:101DAC002B2826D02C2829D000207047DFF80C02D5
:101DBC00006800687047DFF80402006840687047EC
:101DCC00DFF8F801006880687047DFF8F001006800
:101DDC00C0687047DFF8E401006800697047DFF8FD
:101DEC00DC01006840697047DFF8D0010068C06909
:101DFC007047DFF8C8010068006A7047DFF8BC0163
:101E0C000068406A704700B58BB00A216846FFF73E
:101E1C0089FF0BB000BD00B581B0FEF797FDDFF870
:101E2C00A001DFF8A0110068884218BF00F032F85A
:101E3C00DFF89401B0F5B26F03D001B05DF804EB9C
:101E4C0029E001B000BD00B581B00FF21D00FFF715
:101E5C006DFFFFF763FFFFF76DFFFFF76FFF01B03B
:101E6C005DF804EBFFF76EBF00B581B0FEF7E0FB49
:101E7C00FEF7B6FB01B05DF804EB0320FFF766BF7D
:101E8C0010B504460320FFF761FF2046BDE8104063
:101E9C00FFF760BFFEE7FEE700B581B0FFF75EFF1E
:101EAC00DFF82801C06801B05DF804EBFFF75ABFFA
:101EBC00DFF81C11DFF81C0188617047DFF818117E
:101ECC0001280CBF40F2FF70002008600020704712
:101EDC0030B581B0FFF71AFFDFF800510446E888EF
:101EEC0020B1FFF7BBFE60B10020E880FFF780F85F
:101EFC0005461020FEF7D4FF012D0BD1FFF79DF8FE
:101F0C0008E0052105F13000FEF77AFB05F1300001
:101F1C00FEF77AFB204601B0BDE83040FFF7FABE71
:101F2C0010B5012818D1FFF723FE012816D0FFF7B2
:101F3C007DFEDFF8A8400120E08004F13000FEF7C0
:101F4C005BFB052104F13000FEF75AFB04F1300075
:101F5C00FEF75AFB002010BDFFF7A3FE002010BDBA
:101F6C0010B501240E2805D10120FFF701FE012830
:101F7C0005D003E0DFF86810085C00B900242046A7
:101F8C0010BD00207047FFF7F1BEFFF7F3BE01B99B
:101F9C001449FEF751BB10B588B0044600200190DF
:101FAC000B461820009002AA21460F48FFF7E6FEC8
:101FBC0002A92046FEF7DFFB08B010BDF00100209F
:101FCC0098CA011070472820900500007801002065
:101FDC00440100200004000000000460B80500204B
:101FEC00383E0020448C000008F80100006801070E
:101FFC0001D50420704700F003007047F8B5054682
:10200C007748784C0068800705D50820A071764980
:10201C0076480860F1BD00F0FDF9754A12680021A0
:10202C0012F0030F18BF0121520748BF41F0020103
:10203C000DB141F0040194F90720821A052A02DA45
:10204C00A279914259D0A0F10F0200250023002A59
:10205C001FD402EB02121312082B28BF07231D46B4
:10206C00072D28BF0625634E06EB850756F825502D
:10207C007F687E1BF5B24F0744BFC6F307277D1957
:10208C008F0744BFC6F307477D19CF0748BF05EB41
:10209C001665584E56F82370FEB25FEA417C44BF79
:1020AC00C7F3072C66445FEA817C44BFC7F3074C37
:1020BC0066445FEAC17C48BF06EB1766A2EB0322BD
:1020CC006A434D4B1D681B68A1718032092A9241ED
:1020DC002D17C5F108053427D243DBB27D436B4382
:1020EC0006EBD272B3FBF2F2B2F5803F28BF4FF68B
:1020FC00FF7200F30700A280E07140480068A188DD
:10210C00206000201F2904D21F21A18004E049086F
:10211C00401CB1F5007FFAD20F39090940EAC10021
:10212C00314A37490843106000205060F1BD10B5AA
:10213C003448006884B224B300F06CF9294991F951
:10214C000720904205DA6FF07F029042B8BF10462C
:10215C00C8718888844201D28C8010BD274A1268CD
:10216C000B68D21A921C202A28BF1F22231A52084D
:10217C0023FA02F42018B0F5803F28BF4FF6FF7009
:10218C00888010BD2048006800B9704710B41F4902
:10219C008A6802F04063B3F1406F1ED04B689B0716
:1021AC001BD40F4B1C680968C1F303511C31090186
:1021BC0014F0050F06D088420FD224F005001860E9
:1021CC0010BC7047814208D2100158BF44F0010482
:1021DC00500158BF44F004041C6010BC7047000050
:1021EC0000000940D43E002030100940FDFDA40041
:1021FC00242208409C130050B43F00500820094092
:10220C0000FFA4803410094028500940AC3F005016
:10221C00EFF3108072B67047EFF3108062B6704720
:10222C000138FDD1704770471B4213D1094236D19A
:10223C002AB18446B0FBF2F002FB10C2704700F0EA
:10224C00FDB8FCD30022002370470B0002000021D4
:10225C0000207047904271EB030CF6D370B5B1FAC5
:10226C0081F4B3FA83F52C1BA340C4F1200532FA98
:10227C0005F63343A2405FF00046E64002E05B08FF
:10228C005FEA3202841A71EB030524BF204629460B
:10229C007641F4D302000B003000002170BD012AFE
:1022AC00CFD970B5140C20D0B1FA81F4B2FA82F502
:1022BC00C4F120046419B4F12006D6D3B2405FF007
:1022CC000044F440002502E052085FEA3303C61ACA
:1022DC0071EB020E24BF3046714664416D41F3D35D
:1022EC0002000B002000290070BD0C46B1FBF2F17E
:1022FC0002FB11452D0445EA1045B5FBF2F402FB37
:10230C00145580B240EA0545B5FBF2F002FB1052C1
:10231C0040EA044070BD000038B5FFF779FF06496C
:10232C000C684D68401E8041C00F18BFFFF774FF4A
:10233C00280C40EA044032BD082009402D480068B2
:10234C00000C00F00700032828BF4FF0FF30704747
:10235C0029490968C1F30F314BF69A1291424FF09B
:10236C00FF3001D1002070474BF6BE12914201D1D3
:10237C00012070474BF62032914208BF0220704773
:10238C0010B41D491D4B0A681B680968120FDBB29B
:10239C00802B28BF0023C1F30F314BF69A14A142B6
:1023AC004FF0FF300CD1012A08D0032A1DD0072A88
:1023BC001DD0082A08BF03F1160013E00A2011E013
:1023CC004BF6BE14A14206D1002AF7D0022A09D13D
:1023DC0003F1140006E04BF62034A14204BF002A9E
:1023EC0003F10A0010BC40B270471420FAE7152024
:1023FC00F8E700009412005018130050A010005081
:10240C0080B5FFF7A5FF18B9FFF7BAFF162800DA59
:10241C00FEE701BD0748084A816812780068C903C5
:10242C0052B2A0F54070C9135043A1EB201080307C
:10243C0000127047285009400C13005070470000E0
:10244C002DE9F04FA1B08246002016461D460291A0
:10245C000B900DF144086FF000490AE016F8011BCF
:10246C000298D0470028029000F0B9820B98401CCB
:10247C000B903078010001D10B98B2E22528EDD1F8
:10248C000020059006900790089009900A9001E0B2
:10249C0040F0010016F8011F2029F9D023290DD096
:1024AC002B2904D02D2906D030290AD00CE040F07D
:1024BC00020080B2EEE740F00400FAE740F00800BA
:1024CC00F7E740F01000F4E72A290ED129682960BB
:1024DC0051F8042B2960002A0D9204D5514240F08A
:1024EC0004000D9180B2761C11E000210D9109E0E1
:1024FC000D99494505D001EB810302EB43013039BD
:10250C000D91761C3278A2F130010A29F0D3317882
:10251C002E2903D04FF0FF310C911DE016F8011F4E
:10252C002A2907D129682960761C51F8042B2960C7
:10253C000C9211E000210C9109E00C99494505D051
:10254C0001EB810302EB430130390C91761C32789C
:10255C00A2F130010A29F0D3ADF838000FF6A840EB
:10256C00317800F05FFE08B116F8010B8DF83A00D7
:10257C009DF83A00682802BF31786829622005D09E
:10258C006C2804BF30786C2803D171208DF83A0088
:10259C00761C11A8049016F8017BB7F125002AD0FF
:1025AC001C3800F0CA80001F022840F2C680133885
:1025BC0000F0ED80093800F0C080801E00F05A81D8
:1025CC00401E00F03081401E022840F2B680001FF1
:1025DC0000F02981401F00F08180401E00F0D78060
:1025EC00401E24D0C01E0BD0801E00F0D080C01E18
:1025FC0000F0CD8048E125208DF8440001204DE10C
:10260C002868286050F8044B286003940C9F002F16
:10261C0004D5204600F012FE074606E03A4600219B
:10262C00204600F027FE00B1071B069737E129680A
:10263C002960002251F8040B29600021CDE900012A
:10264C0011A80390DDE900019142049F08BF90425C
:10265C004FF03C0C01D10C9AC2B100F00F03303397
:10266C00DBB23A2BA8BF2733ACF101020009BB54F3
:10267C00944640EA017009090022914208BF904239
:10268C0004D0039A07EB0C039A42E6D307EB0C0039
:10269C000390CCF13C010C980691814209DA401A66
:1026AC0008904FF6EF71BDF838000840ADF83800CF
:1026BC00F5E0002840F1F3809DF8380000F014009C
:1026CC00102840F0EC800D98059A801A089A801A10
:1026DC00401A0128C0F2E3800890E0E09DF83A002F
:1026EC0062281AD0682806D06A280CD06C281CD016
:1026FC00712808D019E02868286050F8041B28605D
:10270C000B980880CBE02868286050F8042B2860D0
:10271C000B98C117C2E90001C1E02868286050F885
:10272C00041B28600B980870B9E02868286050F8E2
:10273C00041B28600B980860B1E02868C01D6FF07E
:10274C00070101EA00022A60D2E9000108322A607E
:10275C00CDE90001002902D505982D210AE0BDF82C
:10276C003800810702D505982B2103E0C00705D559
:10277C000598202108F80010401C059011A8059917
:10278C00084403903946684600F0ECF987E09DF860
:10279C003A006C280FD0712818BF6A280BD1286812
:1027AC00C01D6FF0070101EA00022A60D2E90001A6
:1027BC0008322A6005E02968296051F8040B296069
:1027CC000021CDE900019DF83A00682803D1DDE92C
:1027DC00000180B20BE0622803D1DDE90001C0B238
:1027EC0005E0742818BF7A2804D1DDE90001002126
:1027FC00CDE900019DF83800000732D5DDE9002352
:10280C000020834208BF82422BD047F0200078285A
:10281C0027D10598302108F80010401C411C059167
:10282C0008F800701DE09DF83A00294600F0DCF82D
:10283C00CDE90001DDE9002300218B4202DA059885
:10284C002D210AE0BDF83800810702D505982B210F
:10285C0003E0C00705D50598202108F80010401C9E
:10286C00059011A80599084403903946684600F074
:10287C00F3F814E0012005902868286050F8041B38
:10288C0028608DF844100AE025208DF844000120C2
:10289C000590380003D088F80170022005900D983F
:1028AC000599401A0899401A0699401A0999401A34
:1028BC000799401A0A99471A9DF83800400710D416
:1028CC002020012F8DF840000BDB3C46012310AA81
:1028DC006946504600F081FC002840F08080641E60
:1028EC00F4D1DDF814B0BBF1000F11AC0CD014F81E
:1028FC00011B0298D0470028029070D00B98401C06
:10290C00BBF1010B0B90F2D130208DF84000089CEC
:10291C00012C09DB012310AA6946504600F05DFC2E
:10292C0000285CD1641EF5D1DDF818B0039CBBF116
:10293C00000F0CD014F8011B0298D047002802900D
:10294C004DD00B98401CBBF1010B0B90F2D13020F9
:10295C008DF84000099C012C09DB012310AA694663
:10296C00504600F03AFC002839D1641EF5D103988A
:10297C000699DDF81CB04418BBF1000F0BD014F80D
:10298C00011B0298D047029048B30B98401CBBF136
:10299C00010B0B90F3D130208DF840000A9C012CD8
:1029AC0008DB012310AA6946504600F016FCB0B9AA
:1029BC00641EF6D19DF8380040077FF55AAD2020F3
:1029CC00012F8DF84000FFF654AD012310AA694683
:1029DC00504600F002FC10B97F1EF6D149E54FF0CD
:1029EC00FF3021B0BDE8F08F622827D068281ED0B8
:1029FC006A2808D06C2828D0712804D0742824D0D8
:102A0C007A280DD021E00868C01D6FF00702104035
:102A1C000860D0E90023083008601946104670475A
:102A2C000A680A6052F8040B0A60002170470A68B1
:102A3C000A6052F8040B0A6000B20BE00A680A60E4
:102A4C0052F8040B0A6040B204E00A680A6052F8BB
:102A5C00040B0A60C11770472DE9F343054608467D
:102A6C002F696F2808BF082405D041F02001782970
:102A7C0014BF0A2410243C26D5E90023642818BF6F
:102A8C0069289046994606D100218B4203DAD8F189
:102A9C00000869EB49090020814508BF80450CD12D
:102AAC00286B50B9082C38D195F83800000734D56C
:102ABC0030203B2687F83B002FE0701E0090064626
:102ACC00404649462246E317FFF7AEFB02F13000C1
:102ADC00C0B23A2803DB9DF8041051390818B855D8
:102AEC00494640462246E317FFF79EFB804689463F
:102AFC000020814508BF804503D0E868B919884299
:102B0C00DBD3082C09D195F83800000705D5B85D42
:102B1C00302802D0761E3020B855B919E960C6F1BC
:102B2C003C00296BA861884208DA081A28624FF623
:102B3C00EF71288F08402887BDE8F38300290ED554
:102B4C0095F8381001F01401102908D1696B6A69E5
:102B5C00891A2A6A891A0E1A012EA8BF2E62BDE89C
:102B6C00F38300002DE9F24F04468EB0D4E9000146
:102B7C00CDE9020104AF9DF8380040F0200BBBF109
:102B8C00610F0AD0206B002848BF062004D408BF70
:102B9C00BBF1670F01D1012020636168C1F30A50BA
:102BAC0040F2FF7290421CD1080304BF2068002839
:102BBC0009D10320A0619DF8380061381A2835D35B
:102BCC000FF2586108E00320A0619DF838006138CD
:102BDC001A2828D30FF23C61E068032200F076FB40
:102BEC00C3E1012815DA204600F0ABFB012810DB0D
:102BFC0000250020BBF1610F1FD1E16830220A7063
:102C0C008A1CE2609DF83820612A0CBF7822582279
:102C1C000FE0626840F2FE3161F31E52451A6260A9
:102C2C004FF0FF30E6E70FF2E851D5E70FF2E8512D
:102C3C00D2E74A706169891C616110B900260025D0
:102C4C008AE1BBF1610F40F09880206BD4E900ABB6
:102C5C0000284CBF2126461CDDE90201002200237E
:102C6C0000F092FB36B23ABF8BF00040CDE902A0E7
:102C7C00CDE902AB06F101082D1FB8F1010F8DF85B
:102C8C0010200DF1110736DBDDE9020100220023D3
:102C9C0000F092FB2FD21C2102A800F0A5FBDDE96D
:102CAC00020100F027FCA8F10708B8F1010F8146DA
:102CBC0009DB00F04BFC02460B46DDE9020100F09B
:102CCC005DFCCDE90201F81D072105E009F00F02BA
:102CDC0000F8012D4FEA2919B9F1010F01DB491E4A
:102CEC00F4D5491E5CBF002200F8012DF9D5C71D93
:102CFC00B8F1010FC8DA0DF11100391AB142B8BFA1
:102D0C000E4636B230000DF111072FD4884206DA88
:102D1C0004A9014449780829A8BF0F2100DA002131
:102D2C0004AA024400E0761E12F80139401E8B42C0
:102D3C00F9D00F2904D104A901444A78521C4A70D5
:102D4C00002802D504AF761C2D1D36B2701E0DD492
:102D5C0039180A783032D2B23A2A03DB9DF838306F
:102D6C003A3B9A18401E01F80129F2D5206B002835
:102D7C0040F1F280701E2063EEE0DDE902010022DA
:102D8C00002300F001FB3CBF81F00041CDE90201C2
:102D9C002DB247F2975068434D49DFF8389180FBCC
:102DAC0001214D1305EBD5752DB2C5F1070ABAF10A
:102DBC00010F98461CDBDDE902675FEACA7007D594
:102DCC0042464B463046394600F098FC06460F46C4
:102DDC004046494642464B464FEA6A0A00F08EFC92
:102DEC00BAF1000F80468946E7D1CDE9026724E0AD
:102DFC00CAF1000A0026384F14E05FEACA7007D502
:102E0C0042464B463046394600F078FC06460F46A3
:102E1C004046494642464B4600F070FC4FEA6A0A6F
:102E2C0080468946BAF1000FE7D1DDE9020132464E
:102E3C003B4600F035FDCDE90201BBF1660F216B7D
:102E4C00DFF898900CBF05F10A0006204618142EE6
:102E5C00A8BF132630208DF810000DF11107012E9C
:102E6C0040DBDDE9020100F05BFB07F10801042205
:102E7C001B4FA0FB0773DB0803EB8307A0EB47009A
:102E8C00303001F8010C164FA3FB0770C00800EBA3
:102E9C008007A3EB47033033521E01F8023DE7D104
:102EAC00083E012E01F10807D9DBDDE9020100F033
:102EBC0037FB00F055FB02460B46DDE9020100F042
:102ECC005DFB00224B4600F019FCCDE90201C8E77E
:102EDC0089B5F814000024400000F03F84D79741D6
:102EEC00CDCCCCCC0DF11100381A0DF1110702E04C
:102EFC00401E6D1E7F1C39783029F9D0BBF1660F4E
:102F0C0008BF691C04D0BBF1650F0CBF0121002167
:102F1C00226B8E1836B2B042B8BF064636B23100BC
:102F2C001AD4814204DA785C3528A8BF392000DA3B
:102F3C0030207A18521E00E0761E12F80139491E14
:102F4C008342F9D0392802D1785C401C785400298E
:102F5C0002D57F1E761C6D1C2DB29DF83810009585
:102F6C0033B23A46204600F003F80FB0BDE8F08FBC
:102F7C002DE9F043054685B01F46D5F83080012F6A
:102F8C008946164602DA01270FF2942649F02000F2
:102F9C00BDF93040662808BF641C17D0672840F084
:102FAC00848014F1040FC0F28680444580F2838043
:102FBC0095F83800641C000702D44745B8BFB846E2
:102FCC0024B2B8EB040848BF4FF0000824B2E868FC
:102FDC00A969012C27DA4A1C30234354B8F1010F9C
:102FEC0003DA95F83800000703D5E9682E208854D9
:102FFC00521C18EB040FB8BFC8F1000424B2604295
:10300C006862A044B845AA61B8BF4746E868AB6996
:10301C003FB2EF613A463146184400F057F9A8EB3D
:10302C000700A862C2E022469742084418DA3A46E2
:10303C00314600F04BF9A9697918E01BB8F1010F82
:10304C00A961686203DA95F83800000705D5EA68CB
:10305C002E205054E869401CE861C5F82880A5E092
:10306C00314600F033F9A86920183F1BB8F1010F65
:10307C0003DA95F83810090703D5EA682E211154A4
:10308C00401CA8613FB2B845B8BF4746E868AB6979
:10309C003FB23A463119184400F018F9A8693818AB
:1030AC00A861A8EB0700686280E0B9F1610F16D146
:1030BC004FF0700918E0474504DA95F83810090705
:1030CC0058BFB846B8F1010848BF4FF00008B9F135
:1030DC00670F14BF4FF045094FF0650904E0B9F1D3
:1030EC00410F08BF4FF05009A969EB68481CA86153
:1030FC00B8F1010F16F8012B5A5403DA95F8381071
:10310C00090719D5EA68431CAB612E211154B8F19B
:10311C00010F11DB7F1E3FB2B845B8BF4746E868C8
:10312C003FB23A463146184400F0D0F8A869381836
:10313C00A861A8EB07006862E868A969014420004F
:10314C0081F8009003D42B2048708E1C03E02D22B4
:10315C004A708E1C644200270DF1080808E00A2210
:10316C00684600F0C8FC019808F8010B7F1C009C15
:10317C0021B20129F3DA022F06DA49F02000652882
:10318C0004BF302006F8010B4FB9302006F8010BB4
:10319C0007E07F1E02A8C05D303006F8010B012F3E
:1031AC00F7DAE868A9690844301AE86195F838003C
:1031BC0000F0140010280DD16869A9690818696A13
:1031CC000818E9690818A96A0818696B8842BCBF15
:1031DC00081A286205B0BDE8F083F8B504460D4620
:1031EC0016461F46002077B116F8011BA868A047A9
:1031FC00A86030B1E86A401CE86200207F1EF3D161
:10320C00F2BD4FF0FF30F2BD686A6C747A4C00006E
:10321C006E616E004E414E00696E6600494E46006E
:10322C00300000000278C9B28A421AB11CBF10F8F3
:10323C00012FF9E718BF00207047000000F10103CF
:10324C00810704D010F8011B89B18107FAD10268FB
:10325C00B2F10131914311F0803F04BF50F8042FBB
:10326C00F6E710F8011B11B110F8011BFBE7C01AAF
:10327C0070470000C9B2830706D0521E22D310F843
:10328C00013B9942F7D11FE0083A13D302F1040233
:10329C0041EA012141EA014150F8043B121F21BFD0
:1032AC004B40A3F1013C2CEA030C1CF0803FF3D003
:1032BC00C9B2001F083210F8013B521E28BF91EA18
:1032CC00030FF8D818BF0120401E704762B38B075C
:1032DC0008D0521E11F8013B00F8013B00F024808D
:1032EC008B07F6D1830740F0208000BF103A07D33C
:1032FC0030B4B1E83810103AA0E83810F9D230BC2C
:10330C00530724BFB1E80810A0E8081044BF51F8D7
:10331C00043B40F8043BD20724BF31F8022B20F8C1
:10332C00022B44BF0B7803707047083A07D3B1E8FF
:10333C000810083A40F8043B40F804CBF7D2530786
:10334C00E4E730B4436803F000420121C3F31303F4
:10335C004360002B04BF0368002B08D10DE0036809
:10336C00DD0F45EA440444605B000360491E446879
:10337C00E302F4D5C4F31303436043681A43426079
:10338C00084630BC704700004FF4001C1CEB410F8A
:10339C0094BF1CEB430F09E041EA030C50EA4C0CC0
:1033AC0052EA0C0C03D2994208BF9042704714BFEA
:1033BC008B428242704700004FF4001C1CEB410F03
:1033CC0094BF1CEB430F09E041EA030C50EA4C0C90
:1033DC0052EA0C0C03D28B4208BF8242704714BFD6
:1033EC00994290427047000070B504460D466068E3
:1033FC00C0F30A5040F2FF71884207D160680003A5
:10340C0004BF2068002817D0022070BD20B92046C8
:10341C00FFF797FF012866DA012D0FDB40F2FF71F1
:10342C00091A8D420AD36068002847BF00202F4933
:10343C0000202F49C4E90001012070BD4142A9427E
:10344C00616806DA6FF31E51401941EA0050606062
:10345C0040E0401E63684519012205F1350062F316
:10346C001F53352801F00041636003D361600020D5
:10347C00206070BD002015F11F0F04DA2068236056
:10348C000022203562606A4212D0401E25688041BD
:10349C00C2F12003C0439D4045EAD07025686668A0
:1034AC00D54006FA03F32B4323606368D340636073
:1034BC0062680A43B0F1004F626003D80DD12078E6
:1034CC00C0070AD52068401C2060206828B96068B5
:1034DC00401C60604FF0FF3070BD6068884204BFD4
:1034EC0020680028F6D1002070BD00BF0000F0FF5E
:1034FC000000F07FF446400D40EAC120490006D29E
:10350C0000F014F8004248BF6FF00040604700F034
:10351C000DF84FF0004188428CBF0846404260478E
:10352C00400D40EAC120490080F00D8040F0004081
:10353C00490DA1F58061491C05D4D1F11F0154BF7F
:10354C00C840C01770474FF000007047010040F1B1
:10355C000980F446404200F005F851F00041604704
:10356C00010000BF09D0B0FA80F18840C91CC1F538
:10357C008461090501EBD02140057047F0B44FF090
:10358C00004591EA030F44BF6B4000F0BBBA00BF8B
:10359C00841A71EB030604D26E40001BB141121960
:1035AC0073414FF4001C1CEB410F34BF7CEB430602
:1035BC0084E00C0DA4EB1356362E7DDC012E43DC7F
:1035CC0045EAC32343EA525312BFD20292025B086C
:1035DC00240545EAC12141EA5051D2EBC020994162
:1035EC0025D407D1B0FA80F610FA06F164D0002089
:1035FC00203608E0B1FA81F6B140C6F1200220FA7B
:10360C0002F21143B0404FEAF474B4EB465434F078
:10361C0001064FEA74040AD8D6F50016760D04F0AC
:10362C000044F04061FA06F25040F1404840C00AB4
:10363C0040EA415021F0004128BF5FEA500550F1AB
:10364C00000044EBD12137E045EAC323DB0A45EA0D
:10365C00C121C90AB6F120050EDD42EA0242120C64
:10366C00C5F1200603FA06F6EB4042EA06056D4268
:10367C00984161F100010DE062FA06F5F240554007
:10368C0063FA06FC82EA0C02F3405A406D42904108
:10369C0061EB030111F4801F05D1641E620502D099
:1036AC006D004041494121F48011430875F10043FC
:1036BC0050F1000041EB0451F0BC70471CEB410F82
:1036CC0015D223F0004352EA43060BD04FEA4C0CC0
:1036DC00BCEB410F04D80C0D661E342EB7DDEBE7A6
:1036EC00801A994150EA410608BF0021E4E708BF5F
:1036FC001CEB430F28BF6FF00001DDE7B0B581EA8A
:10370C00030C0CF0004C40F2FF7515EA11541DBF70
:10371C0015EA1357AC42AF4239E0E41923EA45539A
:10372C0043F48013C90241F0004141EA505EC702E4
:10373C001100A7FB020200284FF00000EEFB012055
:10374C004FF00001E3FB072118BF42F001024018C3
:10375C0000214941E3FB0E01A4F580640F0302D262
:10376C0052004041494154F101046CDD470872F1AB
:10377C00004250F1000051EB0451A1F580115CBFE7
:10378C0041EA0C01B0BD4CEA05510020B0BD05EA80
:10379C001357AC4214BFAF4241E050EA410E1CBF7C
:1037AC0052EA430E02E061460020B0BD24423C4484
:1037BC001BD15FEA070EF6D0090302BF01460020B9
:1037CC00AEF1140EB1FA81F7AEEB070401FA07FE65
:1037DC000C37C7F1200100FA07F7C8404EEA000E7B
:1037EC0023EA455343F48013A2E733F00043B3FAC2
:1037FC0083F704BFB2FA82FE77440B3FE41BB7F1A8
:10380C00200E2FBF02FA0EF3BB40C7F1200E22FA96
:10381C000EFE38BF43EA0E03BA40641C82E750EA3E
:10382C00410E14BF52EA430E6FF000014FF4001723
:10383C0017EB430F8ABF194617EB410FB5E74CEA5C
:10384C0005510020B0BDD4F10104B4F120070FDA0A
:10385C00C4F12007520828BF42F0010210FA07F504
:10386C0001FA07F7E1BF2A43E0403843E1400FE09B
:10387C00352C98DCC7F1200452EA400220FA07F2FA
:10388C0018BF42F0010231FA07F0A1400A430021AF
:10389C0072F1004250F1000051EB0C01B0BD000080
:1038AC002DE9F04140F2FF7581EA030C0CF0004C5D
:1038BC0015EA11541DBF15EA1357AC42AF42E9E0AB
:1038CC00BC41C1F31301C3F31303801A994143F4B0
:1038DC00801304D2641E4000494180185941C9022A
:1038EC0041EA5051B1FBF3F603FB1611A2FB06752E
:1038FC00D7EBC020A94102D2761E80185941C902CB
:10390C0041EA5051B1FBF3FE03FB1E11A2FB0E75F5
:10391C00D7EBC020A94103D2AEF1010E801859415A
:10392C00890241EA9051760546EA8E2EB1FBF3F6F8
:10393C0003FB1611A2FB0675D7EB8020A94102D21E
:10394C00761E80185941C90241EA50514EEA060EC2
:10395C00B1FBF3F603FB1611A2FB0675D7EBC020E7
:10396C00A94102D2761E80185941C90241EA505130
:10397C00B1FBF3F703FB1711A2FB0735D3EBC02008
:10398C00A94167F100070CBF004247F0010766F33D
:10399C00D5274FEA1E31B80814F5806414DDBD0735
:1039AC0075F1004250EB0E5051EB045111F5801F94
:1039BC005CBF41EA0C01BDE8F0814CF07F6141F045
:1039CC00E0410020BDE8F081BD076D0840EA0E50D3
:1039DC0041F48011D4F10104B4F120060ADAC4F1E7
:1039EC0020060200E04001FA06F3E1401843B24021
:1039FC0015430EE0342C14DCC6F1200445EA4005D6
:103A0C006D0820FA06F2154321FA06F0A1400D4389
:103A1C00002175F1004250F1000051EB0C01BDE8A2
:103A2C00F08100205FEA0C01BDE8F081CFB992185B
:103A3C005B41B3FA83F704BFB2FA82F6BF190B3FAE
:103A4C00B7F120062FBF02FA06F3BB40C7F12006E0
:103A5C0022FA06F638BF3343BA401CB1E419641E8F
:103A6C002FE77F4231F00041B1FA81F404BFB0FA84
:103A7C0080F6A4190B3CB4F120062FBF00FA06F116
:103A8C00A140C4F1200620FA06F638BF3143A0400D
:103A9C003C1B16E7AC421ABF05EA1357AF4214E0C1
:103AAC0050EA41061CBF52EA4306BFE750EA410701
:103ABC00304661461CBF41EA0551BDE8F08152EA2F
:103ACC00430C08BFC143BDE8F08100204FF4001641
:103ADC0016EB410F98BF16EB430F08BF16EB410FC7
:103AEC0024BFC14305E016EB430F0CBF61464CEA03
:103AFC000551BDE8F08191FBF2F303FB1211C0E913
:103B0C0000317047841A71EB030603D2001BB141DC
:103B1C00121973414FF4001C1CEB410F34BF7CEBAA
:103B2C00430443E00C0DA4EB1356352E50DC45EA50
:103B3C00C323DB0A45EAC121C912B6F120050DDD0C
:103B4C0063FA05F6EB4086EA0305124218BF45F00E
:103B5C000105C01851F100010CD213E062FA06F510
:103B6C00F2405540F3415A40B340F3405A4080185C
:103B7C00594107D349085FEA30005FEA350528BF91
:103B8C0045F0010501F58011420875F1004250F134
:103B9C00000041EB0451F0BC4FF4001C1CEB410F36
:103BAC0038BF70470020090D090570471CEB410F09
:103BBC0010D252EA43060BD0BCEB410F05D80C0DCA
:103BCC00AB43661E342EB5DD02E0AB438018594181
:103BDC00F0BC7047F0BC7047DFF800F0D9C10110A1
:103BEC00DFF800F041AC0110DFF800F025B1011056
:103BFC0080B5002804D008233C220021FFF7ECFFFD
:103C0C0001BD3EB504000D000820ADF800000120F8
:103C1C00ADF802006846DFF8E01909688847BDF87E
:103C2C0004102180029929603EBD00B583B00821A3
:103C3C00ADF800100321ADF8021001906846DFF8D2
:103C4C00B8190968884707BD70B584B004000D0029
:103C5C0016000820ADF800000920ADF802006846F7
:103C6C00DFF8941909688847BDF804102180BDF865
:103C7C00061029800299316004B070BD00B583B084
:103C8C000821ADF800100A21ADF802100190684629
:103C9C00DFF86419096888470EBDE0B50821ADF856
:103CAC0000100421ADF8021080B201906846DFF8D4
:103CBC00481909688847002801D0002000E00298C4
:103CCC000EBD00B583B00821ADF800100521ADF88C
:103CDC00021001906846DFF820190968884707BD73
:103CEC00DFF818090068704730B599B0642269464E
:103CFC00822000F072FD6846FFF7A0FA0400601CF9
:103D0C00DFF8FC1808700920DFF8F41848706946D1
:103D1C00DFF8F05822002800FFF7D8FA0922DFF864
:103D2C00E818DFF8DC082044841C2000FFF7CEFAEA
:103D3C0019B030BD00B58FB06846FFF759FFDFF8FA
:103D4C00CC08079040F6C410089001200690002380
:103D5C006A460FF20931DFF8B808FFF745FF0FB0DC
:103D6C0000BD10B58EB0DFF8B018DFF8B008FFF763
:103D7C0048FF00F0C1FD00208DF80800012202A9C7
:103D8C00882000F02AFD9DF8080000280ED00CA811
:103D9C00DFF88C18D1E90023C0E9002306220CA916
:103DAC00812000F01AFD0CA801F0ABFAFFF79CFF84
:103DBC00DFF87018DFF8700801F064FCDFF85418B5
:103DCC000860DFF8680801F0B8FDDFF864180860D7
:103DDC00DFF8600801F0B1FDDFF85C180860102016
:103DEC00019000200090002364220FF27D71DFF817
:103DFC004C0801F057FD06211F2001F0D2F80120DC
:103E0C008DF80E000020ADF81C0001208DF80D007F
:103E1C001020ADF81A001020ADF818000020ADF8F5
:103E2C0016004FF4FA60ADF814000DF10E020121EA
:103E3C0040F2053001F0EAFD07AA022140F20630FB
:103E4C0001F0E4FDDFF8B807FFF7F8F90100DFF83F
:103E5C00B027C9B24FF4427001F0D8FDDFF8E0276B
:103E6C00072140F2073001F0D1FD0DF10D020121C7
:103E7C004FF4447001F0CAFD0DF11A02022140F218
:103E8C00113001F0C3FD06AA022140F2123001F0FC
:103E9C00BDFD0DF11602022140F2133001F0B6FD0A
:103EAC0005AA02214FF4457001F0B0FD1521002246
:103EBC00DFF89047200002F055FA1522DFF884173E
:103ECC00822000F08AFCDFF87C07FFF7B7F90100CD
:103EDC00DFF87027C9B2002000F064FF2020ADF895
:103EEC0012002020ADF8100004220DF112018920DF
:103EFC0000F073FC042204A98A2000F06EFCBDF8CB
:103F0C001210062001F04DF8BDF81010072001F03A
:103F1C0048F8BDF81210082001F043F8BDF8101055
:103F2C00092001F03EF800200B9001208DF80C00C8
:103F3C0001208DF80B0000208DF80A0001208DF86F
:103F4C0009000BAA04214FF4816001F07FF803AA49
:103F5C0001214FF4806001F079F80DF10B02012181
:103F6C0040F2024001F072F80DF10A02012140F218
:103F7C00034001F06BF80DF10902012140F20640FB
:103F8C0001F064F85FF0FF3000F009FF5FF0FF30E4
:103F9C0000F0CEFE02F01AFA5FF0FF3002F020FBC8
:103FAC00DFF8A40602F047FBDFF8A00601F002FFE1
:103FBC00DFF89C0600F080FE5FF4E1300A900320ED
:103FCC0009900020089008AA09A90AA800F064FB2F
:103FDC000A98DFF8801688610998DFF87816087758
:103FEC000898DFF870164877DFF8680602F033FCA3
:103FFC00DFF828060088C0B200F05BFEDFF81C0674
:10400C000088C0B200F0B1FE0FF2755002F0BBFD9B
:10401C000FF26D5002F00AFC20200190002000905D
:10402C0000234FF47A720FF24151DFF82C0601F0A5
:10403C0039FC0020009001226946862000F0CDFB5F
:10404C000098002807D0DFF8100601F04FFC002183
:10405C00082002F01BFE0EB010BD000010B584B09D
:10406C00FFF77FFE8EE0DFF8C805006801F090FCDA
:10407C000400002C05D0200000F0C7F92000FFF749
:10408C0020FEDFF8AC050068FCF7C2FA0028EAD085
:10409C00DFF8C805007840070AD5DFF8C0050088AE
:1040AC004FF6FB710840DFF8B415088000F05BFA9E
:1040BC00DFF8A8050078800664D5DFF8A40502F0C7
:1040CC009DFDDFF8980500884FF6DF710840DFF89A
:1040DC008C150880DFF88C05007806284ED0DFF8A8
:1040EC0084050078072849D0FDF718FEDFF878051D
:1040FC0002F084FD0120DFF87415096849688847CF
:10410C0046F2CE410120DFF864251268526A9047CE
:10411C00FFF7E6FDDFF85805FEF782F80420FCF700
:10412C00B3FC0820FCF7B0FC002200210120FCF7B6
:10413C00ABFD0420FCF78AFD0820FCF787FDDFF8B7
:10414C003005FEF76DF80620FCF770FC0920FCF733
:10415C006DFC01208DF8040001AA012140F205300C
:10416C0001F054FCDFF8EC0402F075FB4FF4FA504C
:10417C00FEF756F8DFF8FC0402F040FDDFF8F80417
:10418C0002F03CFD5FF0FF30FFF778FD00287FF474
:10419C007FAF002000906A4602A90DF10600FFF7E0
:1041AC0053FD002824D10124BDF80600102816D197
:1041BC00BDF80800DFF86414098888420FD1009814
:1041CC0001884FF6FF72914205D18078000706D521
:1041DC0000F0D5F803E0009800F0A1F80400009876
:1041EC00002805D0E4B2002C02D00098FFF71DFD8A
:1041FC00DFF844040068FCF70BFA00287FF441AFA9
:10420C00DFF834040068FCF70BFA8468002C3FF4E8
:10421C0038AFDFF868040078012855D1DFF8440482
:10422C000078062804D0DFF83C04007807284BD12E
:10423C000120207810280ED0202844D1601CC0B258
:10424C0002F034FADFF8F003006801F0A1FB200063
:10425C00FFF737FD15E7627DDFF82414601C02F0D0
:10426C0043FD002809D10020DFF81014087000214C
:10427C00002002F00BFD002004E0621C617D002098
:10428C0002F0E0F9C0B2002804D0DFF8F80301F026
:10429C002DFB17E0607D80B202F0FDF9DFF898038A
:1042AC00006801F075FBDFF890030068FCF7B0F9CB
:1042BC00002804D1DFF860030068FFF791FC2000B0
:1042CC00FFF7FFFCDDE6DCE6627DDFF8B413601C73
:1042DC0002F00AFD002808D10020DFF8A0130870B6
:1042EC000021002002F0D2FC03E0617D601C02F092
:1042FC00ABFD607D80B202F0CEF9CF48006801F0D2
:10430C0047FBCD480068FCF783F9002803D1C2486D
:10431C000068FFF765FC2000FFF7D3FCB1E680B521
:10432C00010001200A78912A05D0B02A07D1080093
:10433C0000F007F803E049780E29FFD0FFE7C0B280
:10434C0002BD10B50400607816280FD10822B348BE
:10435C000188C9B2608800F0DCFF002808D1012078
:10436C0000F038F8C8480460002007E020797E2867
:10437C00217914F1080000F0B7FE012010BD10B532
:10438C00C1480068002824D0C0480078401CBF49B0
:10439C000870BD48006810F10802BB48006801793C
:1043AC00B9480068408800F0E8FC0400E4B2162C20
:1043BC000FD0E4B2042C0CD0002298480188C9B26A
:1043CC00B1480068408800F0A4FF2000C0B200F0A3
:1043DC0001F810BD80B5AC490968002914D0C0B2F1
:1043EC00002807D0A84800680179A7480068083061
:1043FC0000F07AFEA4480068FFF717FC0020A249E1
:10440C0008600020A149087001BD80B50188012910
:10441C0002D0022904D007E0807800F00DF803E008
:10442C00807800F08FF8FFE701BD80B50100C9B2BC
:10443C00012000F0CDF801BD10B58AB00400E4B243
:10444C00200001280AD0022842D0042856D0052882
:10445C005FD006283DD007284FD068E006A802A9F7
:10446C004FF4417001F016FC9DF808008DF8000027
:10447C009DF809008DF801009DF80A008DF80200E6
:10448C0000208DF8040000208DF803009DF80D002D
:10449C008DF807009DF80C008DF806009DF80B00B8
:1044AC008DF805006A460821002001F097FF02A84C
:1044BC0001F07DFA0100764802F0A0FB02A906A8E3
:1044CC0000F023F90C2206A9812000F04AF92EE015
:1044DC002DE004A940F2153001F0DCFB0120674906
:1044EC00087004A801F063FA0100052002F0CEFB6D
:1044FC000021072002F0CAFB19E018E01420FFF796
:10450C0069FF00205D4908700021062002F0BEFB07
:10451C000DE01420FFF75EFF0020584908700021C1
:10452C00092002F0B3FB0021062002F0AFFB4D483E
:10453C0004700AB010BD80B50100C9B2022000F0B1
:10454C0047F801BD10B586B004006846142102F08E
:10455C00D3FDE4B2002C04D16946002002F0C5F86A
:10456C00FFE706B010BD704780B53C490988084389
:10457C003A49088028480068FFF732FB01BD00006B
:10458C00F8B505000E0014001620FFF786FB070097
:10459C00002F1CD016210022380001F0E3FE3D70E4
:1045AC00E4B27D1C220031002800FEF78FFE7C75E2
:1045BC003A00194801682048006801F0C5F9012843
:1045CC0005D134480068E4B2001B32490860F1BDE3
:1045DC0038B504000D000420FFF75FFB002809D05C
:1045EC00E4B20480857002000B4801681048006832
:1045FC0001F0AAF931BD0000EC0800202C20094084
:10460C00F83D0020FA3D0020FC080020B8190020DD
:10461C00F03C0020F03E0020F43E00200C3F002037
:10462C00308D000008090020983E0020A43E002098
:10463C00F83E0020B03E0020FC3E0020B03D0020A3
:10464C0028090020B40800209C09002098090020AB
:10465C00C43E00208C3D0020D43D00200E3F0020A5
:10466C00408D0000133F0020488D00008C0100108D
:10467C0080A90300508D0000588D0000153F0020CC
:10468C00388D0000683D0020003F0020143F0020C2
:10469C00D88C0000C03E002070B582B006000D0022
:1046AC0014000020009004226946832000F095F845
:1046BC00009830600020009001226946842000F0B0
:1046CC008CF80098052802D1002028600DE0009895
:1046DC00062802D10120286007E00098072802D1A3
:1046EC000220286001E003202860002000900122B5
:1046FC006946852000F071F80098022802D101204B
:10470C00206001E00020206073BD7EB500F023F82E
:10471C0005240D5D2D090DF803500DEB03060D5D01
:10472C009B1C641E05F00F050C2B7570F1DB002132
:10473C001DF801300A2B06DA30334354491C0C297E
:10474C00F6DB01207EBDA3F10A04062C38BF3733FB
:10475C00F3D300207EBD6A4600230024002538C216
:10476C00704734B59AB004460D46CAB1642A17D2C4
:10477C00A4F18100012815D9801E03D0401E0A28FF
:10478C0010D90DE00A220021284602F05DFD4FF4FD
:10479C00966190FBF1F14FF4966202FB110008B1A7
:1047AC00002018E06421684602F0A6FC01221AA938
:1047BC006846FEF79BFD1A98421C29460DF1010034
:1047CC00FEF784FD6846FEF739FDC1B26A46E0B2D9
:1047DC0000F0DFFD01201BB030BD70B59AB006466D
:1047EC00002000900C461546642101A802F084FCC0
:1047FC00002D6BD0652D69D2B6F1800009D0401E1A
:10480C0012D0401E05D0401E49D0401E0A2856D951
:10481C005CE000F065F800F05CF8009A0DF1050121
:10482C002046FEF753FD51E06A460121812000F03D
:10483C009BFD0098411C01AAC9B2812000F094FD97
:10484C00012101A807E0A3F16102062A3ED2A3F1DF
:10485C0057024254491C009A521C91420EDA435C96
:10486C00A3F130060A2E38BFA3F13002F1D3A3F125
:10487C004106062EE7D2A3F13702EAE7009A00219F
:10488C0009E001AB1344865C13F8013C46EA0313C0
:10489C006354491C921EA942F3D3012017E06A46C7
:1048AC000121832000F060FD0098411C01AAC9B2CF
:1048BC00832000F059FD00F018F8206006E000F0AD
:1048CC000FF800F006F800F010F8208000201AB065
:1048DC0070BD0098411C01AAC9B2F0B200F044BDF1
:1048EC006A460121F0B200F03FBD0A2200210DF111
:1048FC00050002F0A9BC000030B59BB0642101A8F2
:10490C0002F0FAFB6A460121802000F02DFD9DF893
:10491C000000411C01AAC9B2802000F025FD9DF8C1
:10492C0000200FF26C000DF1050102F0DDF920B949
:10493C009DF8000008B1642828DB0024642101A83C
:10494C0002F0DAFB0FF2580000EB041085682846E1
:10495C00FEF774FC8DF8000001A99DF800200A7088
:10496C002846FEF76BFC024629460DF10500FEF7C2
:10497C00ADFC01A8FEF762FCC1B2A4F1800001AA53
:10498C00C0B200F006FD641C102CD7DB1BB030BD90
:10499C00424C455F323031363038303846000000FA
:1049AC0000000000C0F301009C490000040000005E
:1049BC0001000000D0F30100D8F301000400000056
:1049CC0002000000E8F30100F4F301000400000011
:1049DC000300000004F4010014F4010000000000C6
:1049EC00040000001CF401002CF401000000000085
:1049FC000500000030F4010040F40100000000004C
:104A0C000600000044F4010054F401000000000012
:104A1C000700000058F4010040F401000000000001
:104A2C000800000064F4010054F4010000000000D0
:104A3C000900000070F401007CF40100000000008B
:104A4C000A00000080F401007CF40100000000006A
:104A5C000B0000008CF401007CF40100000000004D
:104A6C000C00000094F40100A0F401000000000010
:104A7C000D000000A4F40100B4F4010000000000DB
:104A8C000E000000B8F40100B4F4010000000000B6
:104A9C000F000000C8F40100D4F401000000000075
:104AAC00E0B50821ADF800100190022100F00FF8DC
:104ABC00002814BF002002980EBD00B583B0082159
:104ACC00ADF800100190032100F001F807BDADF81E
:104ADC0002106846DFF87813096808471FB5ADF86F
:104AEC000610ADF804000824DFF864138DF80820D4
:104AFC000393ADF80040ADF802406846096888475A
:104B0C0004B010BD30B585B0144608220291ADF842
:104B1C0000201922DFF8381309680190ADF8022043
:104B2C001D466846884714B1BDF80C10218015B19C
:104B3C00BDF80E102980089A0499116005B030BD9B
:104B4C0000B583B00820ADF800001A2000F014F86E
:104B5C0000280CBFBDF80400FF200EBDE0B5ADF879
:104B6C000000ADF80610002000F006F800280CBF7D
:104B7C009DF80800FF200EBDDFF8D4120968ADF8CF
:104B8C0002006846084750B110F1040F01D104200F
:104B9C00704710F1030F01D10220704701207047BC
:104BAC008123037042EAC111002341F47C41C3709C
:104BBC00818070478223037081800023C3708271CF
:104BCC0070473EB504460820ADF800000D46202085
:104BDC00ADF802001020DFF878120968ADF8040077
:104BEC006846884720B9029810B16FF004003EBDAA
:104BFC0000950023002221464FF0FF30FFF782FF83
:104C0C003EBD10B582B01446CA78012A03D18A88F9
:104C1C00DFF8E8341A8000F010F858B900906946B3
:104C2C002046FFF7CEFF28B900984478FFF745FFE0
:104C3C00204616BDFFF7A7FF16BD0B46022210211A
:104C4C004CE738B51C461546FFF7F7FFC0B9009086
:104C5C0069462846FFF7B5FF90B9009845782800BB
:104C6C0002BF0098C079A04205D1009881680498D1
:104C7C002246FEF72BFB0098FFF71FFF284632BD9C
:104C8C00FFF781FF32BDF8B500F057FA00F0C0F91C
:104C9C0007000DD032462946FFF78CFF00F049F98A
:104CAC003872FFF74DFF3B4601B0BDE8F0403AE0EB
:104CBC00F1BD10220121E6E738B500F0E2F905005C
:104CCC0004D0042200F032F8AC6026E031BD3C8107
:104CDC00BD72FE6034E72DE9F04100F05BF907008E
:104CEC000FD0142200F022F83C72FD603E8287F84F
:104CFC001280FFF725FF3946BDE8F041DFF80024AC
:104D0C007FE72FE038B500F033F8050001D015220D
:104D1C0000E031BD00F00AF82C81FFF711FF2B46A3
:104D2C0001B0BDE8304002221021D7E6012141E755
:104D3C000022042177E02DE9F04100F02BF9070067
:104D4C0010D002220421FFF735FFBC60BD81BE7379
:104D5C00C7F81080FFF7F4FE3946BDE8F041DFF8E4
:104D6C00A4234EE70420BDE8F081102202218AE73B
:104D7C0004460A2094E602211CE7F8B500F07BF902
:104D8C0007000AD01522FFF7F6FFFFF7A0FF394600
:104D9C00BDE8F840DFF8702333E70420F2BD0022B1
:104DAC00032140E000B583B00FF2490301930623C1
:104DBC000093032300F04EF80EBD1078802802BF3C
:104DCC00508840F27F61884208D19088984202BF97
:104DDC0091790098814201D10120704700207047E1
:104DEC0010B582B00624FFE70094FFF7E6FF16BD6E
:104DFC00000000000323F3E71078802802BF5088DE
:104E0C0040F27F6188420CD19088032818BF042897
:104E1C0007D1907901001CBF1028112801D1012065
:104E2C00704700207047F8B500F013FA07000CD05B
:104E3C0032462946FFF7BEFEBC60FFF781FE3946BD
:104E4C00BDE8F840DFF8C422DBE60420F2BD000028
:104E5C00EC0800202DE9F04100F027F807000AD0FB
:104E6C00069A4146FFF7A6FE3C817D81FFF731FF94
:104E7C00079A00F027BA75E74246032190E670B511
:104E8C0082B000F05AF9FFF75BFE1B210091C3B210
:104E9C0032462946204600F0FEF876BD10B582B0A9
:104EAC001D24009400F0F7F816BD04460D46164676
:104EBC0098461020FFF7F4BD2DE9F04180460D46D1
:104ECC0016461F461820FFF7EBFD040014D00022F5
:104EDC0000F05DF800F030FA20726572A672E7609F
:104EEC000698206107986061FFF72AFE2146BDE80D
:104EFC00F0410FF2BD2284E634E70FF2B923112200
:104F0C0000211EE1F8B500F0C0F807000FD00A220E
:104F1C0000F03DF800F00DF838727D813E73FFF71C
:104F2C000FFE3946BDE8F8400FF28D2269E60420E9
:104F3C00F2BD21465020FFF711BE0FF2812306224D
:104F4C0010E12DE9F04180460D4616461F46102013
:104F5C00FFF7A6FD040010D0072200F018F800F0AF
:104F6C00EBF920726572A672E760FFF7E9FD214646
:104F7C00BDE8F0410FF2492243E6F3E60FF2452378
:104F8C0008220021EEE00FF241231022C4E004219C
:104F9C00FFF706BE04460D46164698461420FFF74A
:104FAC007FBD70B500F014F806000BD03022FFF76F
:104FBC00EEFF00F009F83146BDE870400FF20D220B
:104FCC00FFF71FBE042070BD34817581FFF7B8BD9B
:104FDC0004460D460C20FFF763BD30B583B0044684
:104FEC000020ADF8040000F013F805000DD03122BC
:104FFC00FFF7CDFF2C81FFF7A3FD01A90091022340
:10500C000FF2CD122946FFF71CFEBDF804003EBD81
:10501C000A20FFF745BD1CB500208DF8040000F0F8
:10502C0012F804000CD01222FFF780FEFFF788FD67
:10503C0001A9009101230FF29D122146FFF701FEF9
:10504C009DF8040016BD0820FFF72ABDF8B500F046
:10505C0012F807000DD03622FFF799FF3C817D81B5
:10506C00FFF737FE3946BDE8F8400FF27912FFF72B
:10507C00C8BD0420F2BD04460D4616461020FFF7AD
:10508C000FBD04460C20FFF70BBD04460D4616461B
:10509C000E20FFF705BD2DE9F041FFF77BFF070060
:1050AC0011D0069AFFF7E9FE3C813E74FD6000F0DA
:1050BC0043F97874FFF744FD3946BDE8F0410FF22F
:1050CC005912FFF79EBDFFF74DBE38B51446104A76
:1050DC0015682A0006D0009302460B462146012093
:1050EC00A84732BD002032BD0A4A13681A0003D00B
:1050FC000A4601460120184770470000A809002005
:10510C0045520000555200004B520000054E000065
:10511C00DC3E0020E03E00202DE9F04100F00DF8CF
:10512C0098460C20FFF7BCFC070004D000F016F8E2
:10513C003C81BD72C3E0FFF715BE04460D46164612
:10514C0070472DE9F041FFF7B0FE070004D000F0E6
:10515C0005F8BC60FD60B2E0FFF704BE32460421E6
:10516C00FFF71EBD2DE9F041FFF79FFE070006D0AB
:10517C00FFF7F4FFFFF7DDFE3872FD609FE0FFF7ED
:10518C00F1BD1078802802BF508840F27F618842C0
:10519C000CD190884FF680710140B1F57E4F04BF61
:1051AC0000F07F00984201D1012070470020704729
:1051BC000023E6E71123E4E70A23E2E70623E0E70E
:1051CC000723DEE70823DCE71023DAE73023D8E7F0
:1051DC003123D6E780B5122300930123FFF7EDFDB1
:1051EC0002BD00003623CCE71078802802BF50881F
:1051FC0040F27F6188420DD190884FF6807101405A
:10520C004FF68052914204BF00F07F00984201D1CA
:10521C00012070470020704770B5FFF78EFF1D23EB
:10522C00FFF7E2FF30B9324629462046BDE8704010
:10523C001B23D9E7012070BD80B51423CCE780B5C2
:10524C00152300930223C9E780B50223009304239E
:10525C00C4E704460D4616460C20FFF721BC2DE989
:10526C00F041FFF76AFF98460E20FFF719FC070084
:10527C0009D000F01CF83D817E81A7F80C80FFF767
:10528C005FFC069A1EE0FFF76DBD2DE9F041FFF7BC
:10529C0081FE070009D000F00AF8BD60FE60C7F877
:1052AC001080FFF74DFC069A0CE0FFF75BBD8120E8
:1052BC0038700120F870BC8070473D81FE60FFF7AC
:1052CC003FFC42463946BDE8F041FFF79ABC1078E6
:1052DC00802802BF508840F27F61884204BF9088CA
:1052EC00984201D10120704700207047FFF7B7FFAB
:1052FC0002BD00910023014600227047FFF7C5FF55
:10530C0002BD80B50FF24901FFF7F3FF4FF60C40D9
:10531C00F4E738B50446154600F00FF80FF23901E2
:10532C000091C2B22B4621464FF61840FFF797FF6B
:10533C0032BD3C817D81BE8141465020FFF70EBCC1
:10534C0080B50FF21D01FFF7D4FF4FF61D40CDE7DE
:10535C004FF60C43BBE700004FF61843B7E70000CD
:10536C004FF61D43B3E70000F8B5FFF784FE0700C6
:10537C000DD0012200F022F83C727D72FFF7A9FCDF
:10538C003946BDE8F8400FF26D02FFF73ABC042035
:10539C00F2BDF8B5FFF76FFE07000DD0022200F04A
:1053AC000DF83C727D72FFF794FC3946BDE8F8406D
:1053BC000FF24502FFF725BC0420F2BD0521FFF7D3
:1053CC00EFBB1078802802BF508840F27F61884282
:1053DC000DD190884FF6807101404FF6806291425A
:1053EC0004BF00F07F00984201D1012070470020DB
:1053FC00704700000123E4E70223E2E7DFF800F046
:10540C00CDA00110DFF800F0C1C10110DFF800F0F1
:10541C0009B70110DFF800F03DC10110DFF800F012
:10542C0029AF011090FAA0F0B0FA80F0704780B567
:10543C00DFF8F8030068FFF7F5FF0121DFF8F02330
:10544C00814011600121DFF8EC231160DFF8E813D3
:10545C000A6890420BD201EB80014A683AB113689A
:10546C00190004D0C1B21046BDE80440184701BD74
:10547C00F8B50D00ECB244BF85F0204585F4C0456D
:10548C00A10001F1804101F5012100EA05060A683D
:10549C00DFF8A8733E4085EA02038243324303409F
:1054AC0000F4E0261B0EB6F5E02F03F0010302D149
:1054BC00D30105D411E010F4E02F08BF002B0CD061
:1054CC0002F4E023B3F5A02F04D0B3F5C02F04D120
:1054DC00052300E0062363F312420A60410205D55E
:1054EC00A90DDFF85C2301F00101115500020ED566
:1054FC00FCF70CFC00F057F92C024CBF1C460024A6
:10550C009A4322430A60BDE8F240FCF703BCF1BDAC
:10551C00002948BF0021800000F1804000F50120E7
:10552C0001F03F010268920941EA82110160704763
:10553C002DE9F04F97B08146FCF70AFF00250128B2
:10554C0004D1FCF7FBFE022808BF0125DFF8F402AA
:10555C00C168C1F3815101294FF0010A04D10068DF
:10556C00000E0AFA00F00543DFF8DC02DFF8C8622F
:10557C000078DFF8D8020068C0F346003060FCF712
:10558C00E7FE012802D13068401C30603168DFF83A
:10559C00C07219B1FF22384601F080FE4FF00008AE
:1055AC00002405E0CC550AFA00F040EA0808641C17
:1055BC0059F82400C1B2FF2908D03268914203D2B5
:1055CC0025FA00F2D207EDD5022058E00920FBF7AE
:1055DC00E7FAC6F880900823242200210DA8FFF7D3
:1055EC0011FF8DF84CA00DAA012106F1A000FFF7C8
:1055FC000DFF0024DFF85CA20BE05046FFF738FFEC
:10560C004FF0FF31E0B2FFF783FF0020CBF804002E
:10561C00641C3068844212D225FA04F0C00706EBF1
:10562C00840B48BF0420F1D428FA04F0C00747BF0C
:10563C00E05D59F82010E0B240F4C041DDE70823EA
:10564C003022002101A8FFF7E5FE0020009001ABFD
:10565C00DFF80422102106F18400FFF7DFFEDFF8EB
:10566C00FC01016821F47C5141F4005101600120DE
:10567C00DFF8EC110860DFF8EC110860002017B0BF
:10568C00BDE8F08F2DE9F041DFF8AC6104460D4622
:10569C0006F1A00800F032F800273DB90020206088
:1056AC006060A06000271DB31EE07F1C15F827006A
:1056BC00FF28F3D03168884204D206EB80004068A2
:1056CC000028F2D0002413E006EB800101224C608C
:1056DC0002FA00F0616808436060204655F8272004
:1056EC005C4900F078F87F1C15F82700FF28EBD1F7
:1056FC004046FEF775FA2046BDE8F0814FF0FF31C9
:10570C004046FFF77BBE10B50C46F0B1416821FA5C
:10571C0004F2D20719D50122A24091434160002026
:10572C00454901EB840250604948225C4948FF2AF4
:10573C000EBF44F02041D1F8801051F82210FFF731
:10574C0097FE4FF0FF31204668E0022010BD10B5E7
:10575C00044605E0FFF766FEC1B22046FFF7D3FF13
:10576C0060680028F6D110BD3F49096821FA00F2A3
:10577C0002F00100704738B50C462F4915460A68EF
:10578C00944204D201EB84014968814201D0022089
:10579C0032BDFCF7BBFA00F006F89A4305FA04F3A5
:1057AC001A430A603EE031490A680123A34070475E
:1057BC0010B5214B1C68A14204D203EB81035B683A
:1057CC00834201D0022010BD10001D4A18BF0120D9
:1057DC005054002010BD38B5174C25680B461146A7
:1057EC00CAB2AA4204D204EB82025268824201D0AD
:1057FC00022032BD1846FFF73BFE002032BD0B469F
:10580C0010B511460C4A1468A34204D202EB830271
:10581C005268824201D0022010BD1846FFF778FE74
:10582C00002010BDFCF776FA002032BDE0200240CB
:10583C00E020026080E200E0D03B0020007F077F88
:10584C0000200240A83F0050173F00208012084063
:10585C00183E0020007FC7673B5400000030094011
:10586C000C40094008000940C0200240D0200240F2
:10587C00DFF800F085C10110DFF800F0A9C10110BC
:10588C00DFF800F079B5011000B583B00821ADF850
:10589C00001001900521ADF80210684653490968C3
:1058AC00884707BDF0B589B004460D4616461F461D
:1058BC000823242200216846FFF7DAFF0F984C4991
:1058CC00096806906B464FF47A70B0FBF1F101FB5E
:1058DC0007F0059001FB06F20E98ADF81000294672
:1058EC002046FFF7CDFF204609B0F0BDFAF78CBE7D
:1058FC0038B504460D46FAF73CFF10B12046FAF7CE
:10590C007BFE00F013F800FB05F12046FAF778FE59
:10591C002046BDE83240FAF777BE80B5FAF729FF8A
:10592C0000B10120C0B202BDFAF766BE3049096869
:10593C004FF47A70B0FBF1F0704710B504460021BB
:10594C00FAF772FE204610BD70B584B004460820EC
:10595C00ADF800000D460420ADF802000C202349E0
:10596C000968019016466846884758B9029949B1AA
:10597C008E602046FAF750FE15B12846FEF730F936
:10598C00012003E03046FFF77FFF002004B070BD1C
:10599C0010B50446FAF73CFE38B92046FFF76CFF09
:1059AC008468FFF771FF204610BD002010BD30B594
:1059BC0085B0044668460FF240011422FDF796FCB0
:1059CC000C480146A21D062312F8015D2D095B1E31
:1059DC001DF8055001F8015B157805F00F051DF851
:1059EC00055001F8015BEFD105B030BDEC0800208B
:1059FC00808D0000603E0020303132333435363734
:105A0C003839414243444546000000002DE9F04E30
:105A1C00DFF840799246002640F2013B0C467A783A
:105A2C003B7997F803C0B7F81090B0EB0B0540F634
:105A3C007B4132D06D1E38D06D1E3DD0AD1E41D095
:105A4C006D1E00F07B806D1E00F07E806D1E00F0E0
:105A5C008A806D1E00F09A806D1E00F09F806D1E76
:105A6C0000F0A4806D1E00F0AB806D1E00F0B080C5
:105A7C00ED1E00F0B5806D1E00F0BA806D1E00F0BA
:105A8C00BF806D1E00F0C4806D1E00F0C9806D1FBC
:105A9C0000F0D180AD1E2DD0E5E0102C40F0E1805F
:105AAC001022514607F1A40087E0102C6FD1102270
:105ABC00514607F1B40080E0042C68D1DAF80000FC
:105ACC00F862DBE0012C62D1012B35D09AF8000092
:105ADC00F870BCF1000F06D00028F2D1022A19D0C0
:105AEC00052AEED116E00028EBD0012A20D0042A9A
:105AFC001CD11DE0012C4AD1BCF1010F1CD09AF82D
:105B0C00000038715BB1002808D1032A1CBF072A9A
:105B1C00052A03D15FFA89F0FFF730FAAEE00028CE
:105B2C00FCD0012A1CBF042A062A01D0052A02D166
:105B3C00012000F008FCA1E012269FE0022C26D1E7
:105B4C00BAF80000B88299E0202C0DDA07F1CC06E7
:105B5C001F21304601F0C0FB00F093F87C713346F6
:105B6C00224601210DE0202C7BDA07F1EC061F21E7
:105B7C00304601F0B1FB00F084F8BC71334622468C
:105B8C0000215FFA89F0FFF7DCF974E0012C68D191
:105B9C009AF80000052864DAF8716FE0012C60D1E6
:105BAC009AF8000004285CDA387267E0062C58D1A9
:105BBC004FF48670062251463844FDF787FB5DE0B2
:105BCC00012C4ED19AF8000008284ADA787255E078
:105BDC00012C46D19AF80000042842DAB8724DE044
:105BEC00012C3ED19AF8000002283ADAF87245E00E
:105BFC0000F04CF835D1821F8A4232D238833DE016
:105C0C0000F044F82DD1821F8A422AD2788335E0E5
:105C1C0000F03CF825D1B0F5FA7F22DAB8832DE0FC
:105C2C0000F034F81DD1A0F10A0140F67742914200
:105C3C0017D2F88322E0012C04BF9AF80000012847
:105C4C000FD107F18000FFF768FE40B900F020FB90
:105C5C00060013D107F15C00FFF766FE0EE0162676
:105C6C000CE018260AE0272807DA022C05D1BAF82E
:105C7C000010FFF796F9064600E002263046BDE814
:105C8C00F08E224651463046FDF720BBBAF8000094
:105C9C00022C704738B500244FF440730D46C21ADD
:105CAC00DFF8B01636D0521E36D0521E37D0521EE8
:105CBC0038D0521E39D0521E3AD0521E3CD0521EF1
:105CCC003CD0521E3DD0521E3ED0521E3ED0521ED3
:105CDC003ED0521E40D0521E40D0521E40D0921E7A
:105CEC0040D0521E40D0521E40D0521E40D0521EA8
:105CFC0040D0521E40D0521E46D0521E46D0521E8C
:105D0C0046D0921E48D0521E14D0521E42D0521E63
:105D1C0044D046E0887842E01022A43130E01022D2
:105D2C00B4312DE0C86A286042E00622C43127E075
:105D3C00C87834E0087932E0888A36E04A79CC3188
:105D4C001EE08A79EC311BE0C87928E0087A26E05D
:105D5C0006224FF4867012E0487A20E0887A1EE022
:105D6C00C88A22E0C87A20E0088B1EE0488B1CE031
:105D7C00888B1AE0C88B18E006224FF48A70014415
:105D8C002846FDF7A3FA13E0088C0EE0488C0CE0D3
:105D9C00888C0AE0087B02E0487800E0487B287099
:105DAC0006E0272803DAFFF718F9288000E0022420
:105DBC00204632BD1CB5DFF89C45617889B900B12D
:105DCC00206304F12C00019004F1B400009004F164
:105DDC00A403208AA1780022C0B2FFF76DF800203E
:105DEC0016BD112016BDDFF86C054178062918BFC9
:105DFC00072905D1C18A008A1322C0B2FFF782B8E5
:105E0C001220704700B58FB008233C220021684651
:105E1C00FDF7E2FEDFF8400500F150010791002389
:105E2C0040F2EE2108916A46032106910FF2CD0152
:105E3C00FDF7DAFE0FB000BD70B584B000F016F9B6
:105E4C000120DFF81815DFF80C4509680FF2115521
:105E5C00ADF80200002668468847BDF80400208291
:105E6C000298A062002060704FF6FF70E082FFF78E
:105E7C00D2F8207000230120019000220020009015
:105E8C00294604F13800FFF70DFD022000F02FF831
:105E9C0004F15C00FFF706FD042000F028F804F183
:105EAC008000FFF7FFFC0420A07004F1A402002086
:105EBC000021002300252BC204F1B405103A4BC578
:105ECC00E062E0712072A172072060721021022042
:105EDC00FFF74AFA103D2A4610210320FFF744FA37
:105EEC0004F12C0204210420FFF73EFA7FBD01903F
:105EFC00002300200090002229467047FEB5FFF7D2
:105F0C009BFFDFF85054DFF8544405F1800700F094
:105F1C00ADF80A20ADF802004FF0FF300190684652
:105F2C002168884700284BD100F0A0F80920ADF873
:105F3C000200684621688847BDF80610029E0028BA
:105F4C003ED1BDF80400102804BF288A81422DD10F
:105F5C0030884FF6FF71884209D17088400425D5EE
:105F6C0005F12C0204210420FFF713FA1EE030780F
:105F7C00A22805D0D02804BF304600F07BF815E0ED
:105F8C007079132812D13089012804BFA87B02280C
:105F9C0005D13846FFF7C8FCFFF725FF06E00520C2
:105FAC00FFF71BF801463846FFF7A2FC46B100F09C
:105FBC005DF80320ADF80200019668462168884719
:105FCC00688AC10731D54FF6FE7108406882E978BE
:105FDC002879014329D018B103208DF800000DE079
:105FEC00E8798DF800000622287A8DF801004FF42C
:105FFC00867029180DF10200FDF768F9687A8DF8A2
:10600C0008006946A87A8DF80900288AC0B2FEF704
:10601C0094FF00281FBF08206870286B002804D04C
:10602C00016808001CBF08208847688A810706D5CC
:10603C004FF6FD7108406882002000F029F9688A4B
:10604C0041070AD54FF6FB7108406882A87B0128EE
:10605C0004D0022808BFFFF7C6FE58E70090EB8B70
:10606C00AA8B698B288B00F047F950E70820ADF814
:10607C0000007047F8B50546B64CA8784FF48A7105
:10608C006718010004F1800612D002283CD00328C6
:10609C0018BF04285CD0052800F08280062800F088
:1060AC00AD80072800F0CF800F2800F0EB80F1BD09
:1060BC00687801001BD104F1A40210210220FFF723
:1060CC0068F904F1B40210210320FFF762F90622EB
:1060DC00E91C04F1C400FDF7F9F80120607004F12B
:1060EC00CC03208A62790121C0B2FEF72AFF08B1E5
:1060FC0008206070206B30B10168080003D0607814
:10610C00BDE8F4400847F1BD6878E8B9E87848B1D3
:10611C00208AA27904F1EC030021C0B2FEF711FF32
:10612C00687011E06078022818BF07280CD0062888
:10613C0002D12079012807D104F13800FFF7EDFBDB
:10614C0010B9012000F0FFF868780028DBD0CFE709
:10615C00697821BB03280AD16078062808BF07207C
:10616C00C7D0E07800280CBF03200220C1E7A18A29
:10617C000800E07807D0227910430AD004F13800E7
:10618C00FFF7B6FB05E0012807BF0020E0700020F8
:10619C0020716078072814BF04200620A9E7A7E720
:1061AC006878010024D10622291D3846FDF78EF8A7
:1061BC006889E08206206070E8892084288A6084DF
:1061CC00688AA084E8782073E07A012809D11F201E
:1061DC00FEF703FF4FF47A71414304F15C00FFF7C3
:1061EC0087FB6A89E8780423291DFEF774FD81E793
:1061FC003128D4D10020E07004207AE7A888FEF77B
:10620C0081FD0621384601F067F800202084608467
:10621C00A084A879607304F15C00FFF785FB30461D
:10622C00FFF782FB4FF6FF70E082207908B1032064
:10623C005FE7A87908280CBF0520042060700120B6
:10624C0000F081F856E73046FFF76EFB68780028BF
:10625C000AD1E8882084288960846889A08404F1A4
:10626C005C00FFF75AFB00287FF44DAF636B002BEB
:10627C003FF449AF1B68A28C618C208C01B0BDE847
:10628C00F0401847A888BDE8F4400521FEF77BBE16
:10629C00FEB5304D2A8B0446288C904224BF698B66
:1062AC00814207D3688CA98B884202BFA88CE98BEA
:1062BC0088421ED00520FEF790FE0646E88AADF80F
:1062CC000000288BADF80200688BADF80400A88B99
:1062DC00ADF80600E88BADF808006846FEF70DFE39
:1062EC00070007D1AC73314605F18000FFF700FBC6
:1062FC0000E018273846FEBD70B5164C6578062DA3
:10630C0001D0142070BD40F67A45861FAE423CBFCA
:10631C008E1FAE4215D2B2F5FA7F12DAA3F10A053E
:10632C0040F67646B5420CD220836183A283E38388
:10633C000498FFF7ADFF04F15C00FFF7F5FA0020BD
:10634C0070BD182070BD03494A8A10434882886A80
:10635C00FDF746BC38030020802E0020EC080020FE
:10636C00F1E7000062F30F2262F31F42401810F0B5
:10637C00030308D0C91A1FD3DB0748BF00F8012D4F
:10638C0028BF20F8022D130030B4144615461039DE
:10639C0028BF20E93C00FAD8490728BF20E90C00A7
:1063AC0048BF40F8042D890028BF20F8022D48BFB3
:1063BC0000F8012D30BC7047C91818BF00F8012D2A
:1063CC00CB0728BF00F8012D704700000FF2042303
:1063DC007D4810221321FEF7AEBC00002DE9F043DE
:1063EC000024082885B00E469146784F00F28A802A
:1063FC00DFE800F0050C1824303C48537D00082ED3
:10640C0076D13246494607F1080076E0152E77DA48
:10641C00152107F1100000F06FFE3246494607F1D6
:10642C0010006AE0152E6BDA152107F1280000F038
:10643C0063FE3246494607F128005EE0152E5FDA0E
:10644C00152107F1400000F057FE3246494607F18E
:10645C00400052E0152E53DA152107F1580000F0D8
:10646C004BFE3246494607F1580046E0152E47DAF6
:10647C00152107F1700000F03FFE3246494607F146
:10648C0070003AE0152E3BDA88371521384600F0BB
:10649C0033FE3246494638462FE00820ADF8080056
:1064AC000420ADF80A00039602A8DFF82481D8F87E
:1064BC0000108847C8B9049DBDB1786807F1A001E8
:1064CC0088420AD00821ADF8001001900521ADF8E2
:1064DC0002106846D8F800108847324649462846CC
:1064EC00FCF7F4FE7D603E700DE013240BE0072EEC
:1064FC0006D13246494607F1B000FCF7E7FE02E050
:10650C00182400E00224204605B0BDE8F08300000A
:10651C002DE9FE4990464A680A9C107852780B9DEA
:10652C0000EB02201F46002680B242F62322274BA6
:10653C00801A03EB040C07D0401E052810D9801FCD
:10654C001ED0263829D03AE0092C28D2C4F10800F4
:10655C00854228BFC4F108053D800CF1080129E0F3
:10656C00D1F80CB05846FCF769FE80B2A04216DB9D
:10657C00011B8D42A8BF051B3D800BEB040119E0EC
:10658C0018780146A1420AD3001B8542A8BF0D1BF7
:10659C003D8058683A8801190DE0082C01D3072674
:1065AC000FE0C4F10700854228BFC4F107053D8008
:1065BC000CF1B0013A884046FCF788FE01E03E80C1
:1065CC000A263046BDE8FE8908020020540400204B
:1065DC00EC0800201D650000000000000000000019
:1065EC003EB504460820ADF800000420ADF80200CA
:1065FC008349844800780968834D8000019068467F
:10660C008847002814BF002002980100686001D15F
:10661C0013203EBD4FF6FF7000F062FEE00708D578
:10662C000FF2FC131022092105F11C00FEF783FB6D
:10663C003EBD00203EBD00281DBF744908600020EF
:10664C001120704770B584B00C46154600BB152C54
:10665C001CDA6D4E142106F1080000F04DFD2246A7
:10666C00294606F10800FCF731FE0FF29900029062
:10667C003470FF20019006F11C03092000900022C9
:10668C00706806F1080100F045FE02E0182000E0F9
:10669C00022004B070BD0021020004D05C4A1368D3
:1066AC00C018106000E018210846704701285949AD
:1066BC000BD0022805D0082802BF0868401C0860CF
:1066CC0006E08868401C886002E04868401C48600E
:1066DC00002070470021020004D04F4A1368C018F4
:1066EC00106000E018210846704710B50B460024D6
:1066FC0028B9142249491846FCF7E8FD00E00224A9
:10670C00204610BD38B510460A7A0024D20601D5B1
:10671C00082032BD049A0AB10B2032BD0A78102A27
:10672C0012D14A68157B527B05EB022292B24CF2D5
:10673C00E105AA4206D1344A12781A80C968FCF7DE
:10674C00C5FD07E01C8002E0022A1C8001D10A244E
:10675C0000E00124204632BDF0B583B015460A7A1C
:10676C00002492061E4601D50820FEBD0B78089A1F
:10677C00102B2CD14B68187B5B7B00EB032080B279
:10678C004CF2E103984230D11AB9152E03DB0D24DB
:10679C001BE00B2419E0CF681421384600F09CFD57
:1067AC00324629463846FCF791FD3146384600F012
:1067BC00EDF9300018BFFFF78DFF1448006820B1C9
:1067CC00016808001CBF002088472046FEBD022B34
:1067DC0018BF0124F9D14B681C785B7804EB0323B8
:1067EC009BB242F60214A34201D00A24EDE7012326
:1067FC000193009233462A4600F0EFFD0446E4E78D
:10680C00EC080020380300200C050020E43E00209A
:10681C00E83E00208C3E0020EC3E002014050020B9
:10682C0011670000656700000000000072494862B3
:10683C00704738B57148704D0068804704466869E8
:10684C0000F078FE686900F05DFE2046BDE834403B
:10685C006B490968084738B5FFF7EBFF00F05BF8A8
:10686C0004466849002000F053FE63494861002249
:10687C00202100F04AFE00F092F805462046884799
:10688C0000F090F8E8B232BD38B55B4C5D4DE0617C
:10689C002162A261284600F045FE4FF4E130A86168
:1068AC00294600206875A875032028770020687792
:1068BC000120287068700020E8750FF26100E86014
:1068CC000FF219002861002000F022FE6061002206
:1068DC00BDE83840202100F018BE000038B5054650
:1068EC0000F019F804466868434DC07F8DF800002D
:1068FC0030B16B6A180003D00122694620209847FA
:10690C00AA69100002D0698A0020904700F047F86D
:10691C002046884731BD394800680047F8B506461F
:10692C00364800681446804705467068324EC07F72
:10693C008DF8000030B1736A180003D0012269464B
:10694C0020209847CCB1318A002089B2B1F5007F64
:10695C0009DAF769335C7B5400223254401C491C21
:10696C00C0B2A042F1D38442318206D0B269100089
:10697C0009D0718A4FF400709047B269100002D0B0
:10698C000021A0B29047002030821022706931465D
:10699C0000F0CDFD00F003F828468847F1BD1849FA
:1069AC000968704710B5FFF7B6FF0446124900207E
:1069BC0008821022486900F0BAFD2046FFF7EFFF6D
:1069CC00BDE81040084770B504460C480A4E0068F4
:1069DC0080470546316A70697482224600F0ADFD2D
:1069EC00074910F1010F04BF002070820968284686
:1069FC008847708A70BD0000403D0020E4080020EC
:106A0C00E80800208C3D0020DFF800F021B90110CF
:106A1C00E0B500F010F8042100F012F8002814BFC3
:106A2C00002002980EBD00B583B000F004F80521DB
:106A3C0000F006F807BD0821ADF800100190704772
:106A4C00ADF8021068468D490968084730B58C4C82
:106A5C000020A06087B00021FFF7D6FF60600823FC
:106A6C00182200216846FBF792FA4FF4057025189E
:106A7C0069462846FBF78FFAE5600FF2F5120FF224
:106A8C00D9110FF2B51000F06DFD07B030BD70B527
:106A9C007B4C22E020704FF4007104F1140000F0E4
:106AAC002BFB217804F1140000F03CFE2369180044
:106ABC0004D0227804F1140110209847608815281E
:106ACC0003DBE0680121F9F7F3FEA80705D5606840
:106ADC00F9F79EFD08B900F08DF8E0684FF0FF3330
:106AEC000F220021F9F774FE054668071DD5606872
:106AFC00F9F78EFD98B900F04FFD80B96068FEF78C
:106B0C00BBFE06000BD0B1684868A060497800F065
:106B1C007DFDB068FFF787FF3046FFF784FF6068A4
:106B2C00F9F776FD08B900F065F8E807CDD500F067
:106B3C00EBFD15286080ADDB1420ABE780B5FFF7CB
:106B4C0085FFBDE80140A2E730B54E4C4FF400750F
:106B5C008FB0DD22294604F1500000F09FFB082382
:106B6C003C2200216846FDF737F804F150000790ED
:106B7C0008950220069000236A4643492046FDF7FB
:106B8C0033F80FB030BD3E4908617047FEB504467E
:106B9C000D46FF20FEF7E8FD58BB0820FFF738FF35
:106BAC0006001DD0002030700820ADF80000022037
:106BBC0032490968ADF802000195684688470028FB
:106BCC0014BF0020029870607570706818B12A4666
:106BDC002146FCF77BFB0C20FFF71AFF0746BE6033
:106BEC00307830B9264C60683946F9F715FD00F05D
:106BFC0001F8F7BDE0680421F9F75ABE0EB410B5E0
:106C0C00ADF5806D81B004464FF48061684600F0AC
:106C1C0073FAFFAA10322146684600F0A3FD6846BD
:106C2C00FCF70CFB81B26846FFF7B0FF0DF5806DE9
:106C3C0001B010BC5DF810FB1CB5114CA06830B154
:106C4C00FFF7F9FE0321FFF7FBFE0020A0600221F5
:106C5C00E068F9F72DFE13BD80B580B200F020FD81
:106C6C000748C068BDE804400121F9F721BE0000C7
:106C7C000348C0680821F9F71BBE0000EC0800208F
:106C8C0010340020C0310020496B000038B5044698
:106C9C0000208DF800000D46012269468720FDF783
:106CAC009CFD9DF8000068B1074850F8241025B9E8
:106CBC000FF21800FFF7A2FF31BD2A460FF21800A1
:106CCC00FFF79CFF31BD00000808002041542D4106
:106CDC00422025730D0A000041542D41422025739A
:106CEC002025730D0A00000010B401E0491C521E4F
:106CFC006AB10B7804789C4205D010BC2CBF0120E3
:106D0C004FF0FF30704710F8013B002BEED110BC58
:106D1C00002070470AE0491EC9B2425C413A1A2A67
:106D2C0004D2C9B2425C2032C9B24254C9B2002961
:106D3C00F1D1704702E00268521C026002681278BE
:106D4C000B00DBB29A42F6D0704730B59BB0DFF83F
:106D5C007C03FFF753FF002425E06421002201ADE2
:106D6C002800FFF7FFFA6A46012120008038C0B2E4
:106D7C00FEF7FAFA01AA9DF80000411CC9B22000E6
:106D8C008038C0B2FEF7F0FA0DF10503DFF84003CE
:106D9C00210108444268CE482101405A411CCD488B
:106DAC00FFF72CFF641C102CD7DB1BB030BD30B4AC
:106DBC00C94A1278642A02DB0022C74B1A700022DF
:106DCC0005E0C54B1B785B1CC34C2370521C8A42DC
:106DDC0037D2835CC14CC04D2D786355BF4BBE4C34
:106DEC0024781B5D0D2B07D1BC4BBB4C2478234462
:106DFC0013F8013C0A2B0DD0B84BB74C24781B5D13
:106E0C000A2B0ED1B54BB44C2478234413F8013C17
:106E1C000D2B06D1B0480078401CAF4908700020FB
:106E2C0010E0AE4BAC4C24781B5D082BC9D1AA4B9F
:106E3C001B78002B04D0A84B1B785B1EA64C237030
:106E4C00C4E7012030BC704770B582B004000D005F
:106E5C000020009029002000FFF7A9FF00286AD12C
:106E6C009E4C9D4805789E480068FCF7E7F90100A8
:106E7C00C9B22000FFF74EFF99480068FCF7DEF915
:106E8C000200974801682000FFF72EFF002809D068
:106E9C0000209149087064210022904C2000FFF7DB
:106EAC0061FA48E08E480068FCF7C8F92D1A8D4845
:106EBC000068FCF7C3F92D1A002600E0761CAE42E0
:106ECC0008D287480068FCF7B9F92044805D202877
:106EDC00F4D1350082480068FCF7B0F92900C9B23A
:106EEC002044FFF717FF00261AE07D480068FCF7E6
:106EFC00A5F92A007C4951F836102044FFF7F4FE1E
:106F0C0000280CD176480068FCF798F920442844F6
:106F1C0000906846744901EBC60149688847761CA5
:106F2C00062EE2D300206C490870642100226B4CC1
:106F3C002000FFF717FA73BD38B50400002020219C
:106F4C002000FFF7F7FE206800780D2803D020689A
:106F5C0000780A2802D1FFF7F8FE47E0032259A176
:106F6C002068FFF7C1FE002806D0032256A1206836
:106F7C00FFF7BAFE002839D12068C01C20603021F0
:106F8C002000FFF7D7FE206800F002FC0500A81EC9
:106F9C00082820D201202168C0B20844206020219A
:106FAC002000FFF7C7FE3D212000FFF7C3FE202184
:106FBC002000FFF7BFFE2068FCF740F9821E216815
:106FCC0015F17F00FDF7CDFB00280BD0002103202D
:106FDC00FFF75CFE0AE0B5F10A00062801D2022098
:106FEC00D9E703E000210420FFF750FE31BD30B596
:106FFC009BB002242FE06421002201AD2800FFF792
:10700C00B1F93348210108448068FCF717F98DF871
:10701C0000000122694601AD2800FCF757F92C4805
:10702C00210108448068FCF709F92949220111441F
:10703C0089680DF1050502002800FCF747F901A845
:10704C00FCF7FCF801AA0100C9B220008038C0B2DC
:10705C00FEF79FF9641C102C02DA082CCBD1F9E74F
:10706C00002000F006F81BB030BD80B5FEF7BBFE6B
:10707C0001BD80B50020FEF763F900210120FFF768
:10708C0005FE01BD80B51948FEF730FC0021082033
:10709C00FFF7FCFD01BD80B515480078062803D02C
:1070AC0013480078072807D10120124908700021E5
:1070BC000720FFF7EBFD03E000210620FFF7E6FDBC
:1070CC0001BD00007661720056415200B8F6010015
:1070DC00AC4900005C8C0000123F00208C3C00206E
:1070EC009009002094090020E8F60100D43D00200E
:1070FC00133F0020153F0020002200F0D3B8000001
:10710C002DE9F04F85B004461E000D4690461CBF7D
:10711C0000203060A14601E009F1010999F8000056
:10712C00A0F109010529F7D32028F5D02D2816BF89
:10713C002B2819F8017B2B27B8F1000F57D4B8F185
:10714C00010F54D0B8F1250F51DAB8F1010F0DDB56
:10715C00B8F1100F04BF99F80000302802BF99F85D
:10716C00010040F02000782814D10EE099F80000BE
:10717C00302818BF4FF00A080CD199F8010040F0E4
:10718C002000782804D14FF0100809F1020901E021
:10719C004FF00808CDF8109001E009F1010999F8B9
:1071AC0000003028F9D00FF2A40B4FF0000ACDF8F4
:1071BC000C908DF808B00AE09DF80810CDF804A0EA
:1071CC00401AC0B2009008FB0A0A09F1010999F8AB
:1071DC000010A1F141001A2838BF20314246584610
:1071EC00FCF748F80028E7D10498484503D105B1CD
:1071FC002C60002025E00FF27C01039811F8081098
:10720C00A9EB0000401A14D4012808DA0098BAEB54
:10721C00000004D30199B0FBF8F0884209D000F0CB
:10722C00BBFA222101600EB1012030604FF0FF3A11
:10723C0003E02D2F08BFCAF1000A0DB1C5F800906C
:10724C00504605B0BDE8F08F002359E7303132339A
:10725C003435363738396162636465666768696AE4
:10726C006B6C6D6E6F707172737475767778797AEA
:10727C000000000000002115110E0D0C0B0B0A0A6A
:10728C000909090909080808080808080707070771
:10729C0007070707070707070700000062F30F221D
:1072AC0062F31F4200B500BF130096469446103996
:1072BC0028BFA0E80C50FAD85FEA417C28BF0CC06C
:1072CC0048BF40F8042BC90728BF20F8022B48BF41
:1072DC0000F8012B00BD00000022FFF747B80000AA
:1072EC0038B54FF6FF74A0420DD10020654A1378D3
:1072FC0098420EDA21F8204001EB80050023401C57
:10730C00AB70C0B2F3E700F0A9F810B10480002113
:10731C00817031BD2DE9FE4F80460026B8F1000F7B
:10732C0082B006D0080004D0180002D0109F38009C
:10733C0001D1022035E00F9C00252CE0EDB2A946CE
:10734C0038F829004FF6FF7188421EBF08EB890AF6
:10735C009AF8020000281DD0029ABDF83810049843
:10736C0000F02AF85FEA000B14D09AF80200C0076C
:10737C0005D500F019F8012100F086F806439AF8BB
:10738C000200800706D500F00FF8022100F07CF80F
:10739C000643F6B26D1C3B490978E8B28842CDD35E
:1073AC00F0B205B0BDE8F08F019700949DF80C2069
:1073BC0038F829005B46704730B5002400E0641CA7
:1073CC00A3B28B4207D2A4B200EB0413DD68954242
:1073DC00F5D1184630BD002030BDF8B504460698EE
:1073EC000D460026F0B9022B1AD11078517800EB1B
:1073FC0001270798C043B9B201420FD1E868016870
:10740C00204600F012F8B9B288420CD0E868016846
:10741C00BAB2204600F00FF8064604E0802602E0DF
:10742C000D2600E00B263046F2BD80B500F016F8B4
:10743C0000B1807802BD70B504460D46164600F0CA
:10744C000DF840B929464FF6FF7000F007F808B95F
:10745C00112070BD04808670002070BD10B5002214
:10746C0000E0521C074C2478D3B2A34207D2D2B20C
:10747C0031F822308342F4D101EB820010BD0020A0
:10748C0010BD0000380300202DE9F04186B00D46F8
:10749C0090461F46044603AB4FF6FF721B21FDF7C7
:1074AC0014FE059040B3FF2102910246BDF80C106A
:1074BC00DDF834C001910DF112030021009120463A
:1074CC003946E047064688B97889ADF81000E807D8
:1074DC0005D5424604A92046FDF7D1FC05E00C9BDE
:1074EC00424604A92046FDF7D9FC06462EB11B21C5
:1074FC0004A8FDF7F9FD00E01526304606B0BDE8FE
:10750C00F081000001680968084703685B68184748
:10751C00034A0C2303FB00200268D26810470000CA
:10752C0078F701000FF218012422FBF7DFBE036885
:10753C001B6918470168896908470368DB691847A4
:10754C0000000000FFFFFFFFFFFFFFFF0000000037
:10755C00000000000101010100C201000300000055
:10756C000000000070B504464A4800680D4680478C
:10757C00064649480FF22902C4604FF406710561B2
:10758C0001441830FFF780F9FFF70CFA3046BDE8DC
:10759C0070404249096808473F480078704700002E
:1075AC0038B50C463C4D0021A9806880010003D001
:1075BC0029690A0018BF8847200008D000202870CD
:1075CC00E968080003D0E88808B920468847E988AC
:1075DC00080003D06869BDE8344017E031BDF8B548
:1075EC0004460D4600F047F8A84202D200F043F8DA
:1075FC000546294EB788F01900F118012A46204695
:10760C00FBF764FEE819B0802846F2BD2DE9F04185
:10761C0004462048204E0068204F0D468047804687
:10762C00307820B1396840468847002021E0B5F514
:10763C00007F07DD4FF40070A5F5007120444FF476
:10764C00007500E00021F18070612A464FF406704D
:10765C0021463018FBF73AFE01203070B068401C10
:10766C00B0602846FFF7AFF90546396840468847B1
:10767C002846BDE8F081084841888088081A00F542
:10768C000070011200EBD1514912A0EB412080B2E5
:10769C0070470000E4080020682A0020E808002059
:1076AC00F8B52D4C2D4F05466068281860600026F3
:1076BC0060884119B1F5007F08DDC0F50076B1B2E4
:1076CC003818FFF78CFF0020AD1B6080A9B26088D2
:1076DC003844FFF784FF60882288281880B2010A9A
:1076EC0000EBD151490AA0EB4120608075196188EB
:1076FC0040F23910891A8142B9BF61688142184839
:10770C00FEF7F4F8A8B2F2BD134841880088081AB5
:10771C0000F50070011200EBD1514912A0EB412091
:10772C0080B2704770B50C4B0C4D1C8800220CE0DD
:10773C00A4B2521C2E5D00F8016B641CA4B2260A84
:10774C0004EBD656760AA4EB462496B28E42EFD3BF
:10775C001C80084670BD0000BC3E0020383600205E
:10776C00683D002016B504460A46009401AB6946F4
:10777C00064878441630FAF763FE009A002111701F
:10778C0000285CBF0098001B16BD00BF97A3FFFF2D
:10779C000A220021FFF758BD014800F003B8000091
:1077AC00A409002070470000DFF800F0ADB501100F
:1077BC00DFF800F019AE0110DFF800F085C20110FF
:1077CC00DFF800F081C20110DFF800F055C10110A4
:1077DC00DFF800F043C20110DFF800F079AB0110C4
:1077EC00DFF800F0D9B60110DFF800F0EDB30110AE
:1077FC0020B108232C220021F9F78ABE704720B152
:10780C0008233C220021FCF7E7B9704780B5F8F754
:10781C00E7FEADF80000FAF779FAADF8020000982F
:10782C0002BD01B5BDF80200FAF774FABDF800000C
:10783C00BDE80240F8F7D8BE38B5DFF87448DFF879
:10784C0074580020A4F8FC0FE820208040F6147037
:10785C00A4F8E80004F1E8006860002000F003F8E8
:10786C00A8606C6031BDF8B500240025061D16F02B
:10787C0003001CBF311D0E1AFFF7C8FFDFF83428B8
:10788C00B6B21060112EB4BF576897683A881304CB
:10789C0003D582F4004200251AE02B0014D0238873
:1078AC0039880B4423809BB2B34211D327461A4626
:1078BC00B7B1921B92B2042AA7BFBA5346F4004147
:1078CC00398841F4004109E0B242F1DA01253C4625
:1078DC0017443A88002ADAD1002701E027F8041B64
:1078EC00FFF79FFF3846F2BD10B50446FFF78EFF39
:1078FC00DFF8C017086034F8042CC2F30E0224F829
:10790C00042C221F4B689A4238BF4A60BDE81040D5
:10791C0087E738B50446FFF779FF00210C23DFF821
:10792C0098274B43D518AA6C4AB1944204D1FFF75F
:10793C0078FF05F1480032BD491C0329EED3FFF74F
:10794C0070FF002032BD70B50546FFF75FFF04469F
:10795C0000200C22DFF8601742438E18B16C49B935
:10796C0000203065B5640022FFF71EFFF06418B9E3
:10797C0017F040FB8D4205D12046FFF752FF06F170
:10798C00480070BD401C0328E3D32046FFF749FF95
:10799C00002070BD38B50446FFF738FF0025DFF82E
:1079AC0018170C226A438A5A130008D0944203D148
:1079BC00FFF737FFA8B232BD6D1C062DF1D3FFF7D0
:1079CC0030FFFF2032BD10B504462088FFF7E2FFE0
:1079DC00FF2800D16AE10C22DFF8DC165043084482
:1079EC008168080002D16FF0010010BD2046BDE88F
:1079FC001040084702460FF2A470104710B5002043
:107A0C000C21DFF8B426002401FB00F31344401CC6
:107A1C0003289C641C65F7D30020002301FB00F4B1
:107A2C00401C13530628F9D3082010800FF2557010
:107A3C009060BDE81040FFE670B590B0F8F7D0FD4F
:107A4C0004466846FFF7DBFE0520069000224FF443
:107A5C004870089069464FF201000490DFF85C060C
:107A6C000590DFF85C06FFF7A3FE050006D0FFF7D4
:107A7C00CDFE06462846FFF766FF08B917F0BAFA9E
:107A8C003046FFF7CEFE2046F8F7AEFD10B070BDC5
:107A9C00F8B500F0E5F8FFF756FF0546FFF7B6FE20
:107AAC00A28800210C26DFF810364E4333441E8882
:107ABC00370007D11A805D60A2689A60A18169685D
:107ACC002161C4E2B24204D1FFF7ABFE6FF00200B9
:107ADC00F2BD491C0629E5D317F08CFA00BF38B566
:107AEC0000F0BEF8FFF72FFF050016D0FFF78EFE53
:107AFC0000210C23DFF8C0254B431A4413884BB9E3
:107B0C004FF6F8731380556000239360A180696869
:107B1C00A16014E7491C0629EBD317F06BFA00BFE0
:107B2C0010B5044660680C3080B2FFF79CFE10B9AB
:107B3C006FF0030010BD6168018100210160FF211D
:107B4C0081720C30A060002010BD80B540680C38EC
:107B5C0010E080B287E610B50446606880B2FFF78B
:107B6C0082FEA06000280CBF6FF00300002010BD47
:107B7C0080B54068FFF7B8FE002002BD38B504465A
:107B8C000D46FFF743FE002145F80C1C216811B986
:107B9C00256006E0114651F80C2C002AFAD141F868
:107BAC000C5CBDE832403CE62DE9F04104466FF038
:107BBC000206E068A0F10C05E0880628BCBFA0888E
:107BCC0006280BDAFFF722FEE188DFF8EC840C279D
:107BDC0079434144496819B9FFF723FE304617E051
:107BEC00FFF71FFEA0882871E0886871207AA871C1
:107BFC00E088E1687843404440680830FFF7BEFFF6
:107C0C00E0887843404440684068FBF7E9FF002077
:107C1C00BDE8F08170B500F023F8FFF77AFE06009E
:107C2C0002D16FF0040070BDFFF7F0FDB1680025C4
:107C3C0041B10D46A5F10C010A68B26000220A6040
:107C4C00FF228A72FFF7EDFDA560A5F10C010DB9BD
:107C5C00022070BD0879A0804879E080002070BDBA
:107C6C000446F8F7C5BC06280ADA0C23DFF84824CA
:107C7C005843105A02001CBF4FF6F872904202D1C2
:107C8C004FF0FF307047088000207047811D8088BE
:107C9C00E9E710B50446E088FFF77CFEFF2800D129
:107CAC0004E0E0802046BDE810407DE74FF0FF3057
:107CBC0010BD3EB50446FFF7ADFF050017D1A088F7
:107CCC006946FFF7D0FF78B1A06802900821ADF8A3
:107CDC00041001A80321ADF80610DFF8E813896839
:107CEC0088476FF005003EBDBDF80000A080284617
:107CFC003EBD10B5DFF8D02312680C464FF47A71F4
:107D0C00A1FB00010023FAF78FFA002399424FF0F0
:107D1C00004201D8904202D36FF0020010BD2060E7
:107D2C00002010BD38B5FFF79BFFFFF7F2FD0546AD
:107D3C00F8F7B6FC002818BF012800D015B96FF071
:107D4C00040032BD606840B9009000996868FDF786
:107D5C0055FB401E8041C00F32BD10F1010F08BF12
:107D6C004FF0FF30F0D000F04EF90028EDD032BDCE
:107D7C0080B54068FBF734FF002002BD17F03AF9DC
:107D8C0000BF80B54068FFF717FD002002BD80B52D
:107D9C004068FFF715FD002002BD80B5FFF714FD0C
:107DAC00FFF716FD002002BD80B5F8F719FCF9F7B6
:107DBC00ADFF002002BD10B58CB004466846FFF73D
:107DCC0017FDE02000F013F808B917F013F90BE0D9
:107DDC0010B58CB004466846FFF70AFDE06800F069
:107DEC0006F808B917F006F900200CB010BD089081
:107DFC000023A16860686A46FFF7EEBC10B5044624
:107E0C00FFF7EEFC6060002010BD014688684968F1
:107E1C000847F0B507468BB0BC68AA4D6CBB0C206C
:107E2C00FFF721FD04006FF003061ED00823242267
:107E3C00002101A8FDF71CFD0020ADF814000690F0
:107E4C00079400237968A14801AAFFF7CDFC2060B4
:107E5C0068B90820ADF800000C20ADF802006846A7
:107E6C00A96888472046FFF73FFD304618E0F868C0
:107E7C0060603869A060BC600AE0286880470646EC
:107E8C002068F8F7B9FB3869A06030466968884704
:107E9C0079682068F8F7B4FB2068F8F7B5FB002088
:107EAC000BB0F0BD10B5044682B0606800F0ABF8C2
:107EBC0020B9009860602046FFF7ABFF16BD80B577
:107ECC00406810B96FF0020002BD0068F8F794FB2F
:107EDC00002002BD7C49096841600020704750B504
:107EEC000446794802686FF00046A6FB02010023A5
:107EFC004FF47A72FAF798F9002399424FF0004246
:107F0C0001D8904200D330466060002050BD2DE96E
:107F1C00F04186B00646F8F76BFBFFF7FAFC044617
:107F2C00002002900025F8F7BBFB002818BF0128A1
:107F3C0000D014B96FF0040062E0706820B110F149
:107F4C00010F03D14FF0FF30009003E000F05BF81D
:107F5C00070054D1FFF744FC0099012701EB0008FE
:107F6C0000E0009000996068FDF748FA78B303A828
:107F7C00FFF750FE07001AD1BDF8100001A9FFF75A
:107F8C0072FE80B9059ABDF81210BDF80400B368F2
:107F9C00984740B1BDF80400B081BDF81200F081E3
:107FAC000598306113E0059902A8FFF7E7FD0098EA
:107FBC0001276D1C10F1010F18BF0028D2D0FFF75C
:107FCC000FFCB8EB000002D000998142C9D2029E8E
:107FDC00FFF71CFC56B1314600E0114651F80C2C51
:107FEC00002AFAD1A26841F80C2CA660FFF719FC04
:107FFC00002D03E06068FBF7F3FD6D1EFAD13846E7
:10800C0006B0BDE8F081694673E6F8B5FFF728FEC7
:10801C000546F8F745FB002818BF01286FF0040649
:10802C0013D0FFF7F3FB0021234A0C234B43D75A01
:10803C004FB113445B681B68AB4201D1A18006E0D1
:10804C00491C0629F1D3FFF7ECFB3046F2BDFFF7D4
:10805C00E8FB0020F2BDF8B50446F8F721FB002838
:10806C0018BF012802D16FF00400F2BDF8F7C0FA76
:10807C000546FFF7CBFB00210F4A0C234B43D65A86
:10808C0037000ED0A788BE4208D1D11849680968BC
:10809C00A9420CBF01210021A160D8E7491C062987
:1080AC00EBD3FFF7BEFB4FF0FF30F2BD000000003A
:1080BC00B8090020803E00207C23002034080020DA
:1080CC00017A0000E4080020808D0000177E00007B
:1080DC0070B504463C20FFF7C6FB05006FF00306A5
:1080EC0011D0FFF78CFB207AA861002260892862EE
:1080FC002946E06828616068FFF75AFB0446284669
:10810C00FFF7F2FB0CB9304670BD002070BD70B5A6
:10811C0004462420FFF7A7FB05006FF0030613D0DD
:10812C00082324220021FDF76DF92079012808BFCE
:10813C002876A06800222946FFF736FBE060284627
:10814C00FFF7D2FBE06808B9304670BD002070BD67
:10815C0010B5044682B0A06840B9009000996068E0
:10816C00FDF74CF9401E8041C00F16BD10F1010FF8
:10817C0008BF4FF0FF30F0D0FFF745FF0028EDD0DF
:10818C0016BD00004188292902D36FF00100704709
:10819C000FF2140252F8211008470000D3790000A6
:1081AC00197800002F7800009D7A0000EB7A00000F
:1081BC002D7B0000577B0000637B00007D7B000063
:1081CC00B57B0000217C00009F7C0000BF7C000080
:1081DC00317D00007D7D0000897D00008F7D0000D9
:1081EC009B7D0000A77D0000B57D0000C37D0000D5
:1081FC00097E0000B17E0000E17E0000EB7E0000F5
:10820C00997C000085F201004FF301001B7F0000F8
:10821C00178000001F7E0000CB7E0000E9F20100F9
:10822C0021F3010035F301006380000085F30100A8
:10823C00A1F30100DD8000001B8100005D810000C6
:10824C0097F30100AFF30100DD7D0000DFF800F0D3
:10825C0061C20110DFF800F0E1C20110DFF800F09C
:10826C00B9C20110DFF800F0F9BF01108069C00835
:10827C0000F00100704750F8382F1143016070472F
:10828C0050F8382F22EA01010160704741647047B1
:10829C00406800F00F007047002141607047817BFF
:1082AC00FF291CBFC07BFF2801D001207047002094
:1082BC00704738B5F9F72AFDDFF8B457044628782B
:1082CC0020B90420F8F7C2FC012028700CE038B566
:1082DC00F9F71CFDDFF898570446287820B10420E4
:1082EC00F8F7D2FB002028702046BDE83240F9F7A1
:1082FC0011BD40687430FBF773BC40689030FBF7DD
:10830C006FBC70B5446885680E4606E0206A401C58
:10831C002062761E606A401C60624EB1206ADFF8F3
:10832C005427126801782868926990470028EDD18B
:10833C00304670BD70B5456886680C4608E0296B00
:10834C000870641E286B401C2863686B401C6863B3
:10835C0044B1DFF82017096830680969884710F1C3
:10836C00010FECD1204670BD70B504466568A66857
:10837C00FFF7ADFF00F0E2FAD7E270B5446804F104
:10838C00AC050E462846F8F737F90FF24871627FB4
:10839C00207F51F822100818C01D7043DFF8D81642
:1083AC004843A169B0FBF1F0DFF8D01609686430DE
:1083BC00B0FBF1F12846F8F723F92846BDE87040E8
:1083CC00F8F722B9F8B504466568A66805F1AC075C
:1083DC003846F8F711F93068FFF748FF88B1DFF835
:1083EC009C1609684FF4FA70B0FBF1F1022938BF02
:1083FC0001213846F8F704F93846BDE8F240F8F7A1
:10840C0003B9FFF764FF30682021FFF739FF00F054
:10841C0031FA25E270B504460D4620212868DFF8B4
:10842C006066FFF72DFF297B30680122FDF7A3F969
:10843C00297B30680122FDF7BBF9297B30680022CB
:10844C00FDF7DDF9A97B30680022FDF7D8F9A0789B
:10845C00012805D12868FFF709FF0028FAD105E0AB
:10846C004FF0FF3104F17400FCF7C8FF297B306832
:10847C001022FDF7C4F92846FFF711FF30B1A97B94
:10848C003068BDE870401122FDF7B9B970BD2DE917
:10849C00F8438146D9F808603068D9F80470046C48
:1084AC002146FFF7F3FE14F4F06F07F128052DD0E9
:1084BC00600510D53068FFF7EBFE80463068FFF79B
:1084CC00EBFE2969212928BF202100F050F817E084
:1084DC002869401E2861286990B1012100F047F8F5
:1084EC003068FFF7D5FE80463068FFF7D5FEB8F14F
:1084FC00000FEDD0A868401EA860E868401EE86038
:10850C0087F81F80484600F0F9F91FE060060BD58C
:10851C00296900F02CF82861687910B100202861D5
:10852C0011E0286900280DE0E0060FD5287D471ED4
:10853C002869874228BF0746394600F018F8286991
:10854C00C01B286102D14846FFF70EFFA0060CD5D0
:10855C002C6854B121464846FFF7D3FE286020B959
:10856C00211D4846BDE8F44307E7BDE8F1834846C2
:10857C00E0E64068002101700020DFF8F414087078
:10858C007047F0B504466568A76897B00E46F9F7D2
:10859C00BDFB297800294CD101212970F9F7BAFBD0
:1085AC001EB90DA8FEF7BEFF0DAE3078687070785E
:1085BC00A87070686860B068A860F068E86030699E
:1085CC002861307D2875707D6875B07DA875B0699F
:1085DC00A861307F2877707F6877B07FA8770020FC
:1085EC002862286368626863A862A86385F82C0017
:1085FC0085F82D00102085F83C00002085F83D0002
:10860C00B868C0B2F8F7CCFA204600F0A0F92046C2
:10861C0000F0F2F988B9DFF85C1409683868C968A9
:10862C008847B868C0B2F8F74FFAF9F76FFB00212A
:10863C002970F9F76FFB00204DE008233022002150
:10864C0001A8FCF7E7FE00200694009001AB7968C6
:10865C00DFF8302405F15800FCF7E0FE0823242253
:10866C00002101A8FCF7CEFE01208DF81C00A87893
:10867C0040B901AA002105F17400FCF7C7FEDFF830
:10868C0008042861687840B901AA002105F190001E
:10869C00FCF7BCFEDFF8F403E86008232422002179
:1086AC0001A8FDF7E5F800200690ADF8140007943A
:1086BC0001AB0A22DFF8D81305F1AC00FDF7E0F8A6
:1086CC000020009023460FF2D932042105F144001A
:1086DC00F8F751FA204617B0F0BD38B544688568F4
:1086EC00DFF89C030068FDF732F8286840F2F2715D
:1086FC00FFF7C6FDDFF87C1309682868C96888474E
:10870C00A868C0B2F8F7E0F904F15800FFF79EFD35
:10871C00A07818B904F17400FFF79CFD607818B9C3
:10872C0004F19000FFF796FD04F1AC00FFF796FD05
:10873C00F9F7ECFA00212170F9F7ECFA04F1440096
:10874C00BDE83240F8F7A0BB426820296FF0010069
:10875C0002D0212905D07047012082F82D0000207D
:10876C007047002082F82D0070472DE9F84304462D
:10877C006668A7680D469146F9F7C8FA8046B06A54
:10878C0018B14046F9F7C6FA38E006F1AC00F7F735
:10879C0033FF0020F077356270624046F9F7BAFA81
:1087AC00FFF787FDBB48016841F4807101602046EA
:1087BC004946FFF7A6FDB06248B949462046FFF787
:1087CC00DCFDB078F8B900F021F8D0B90DE03868CC
:1087DC002021FFF750FDB078A8B900F017F880B948
:1087EC0049462046FFF7C9FD0020B06239461020EB
:1087FC00F0773046FFF70EFEFFF769FD4FF0FF30C4
:10880C0002E0706A00E00020BDE8F283B16806F176
:10881C007400FCF7F3BD6EE0F8B500F093F8074672
:10882C00A86A40B93068FFF721FD20B93846BDE889
:10883C00F240F9F76FBA0020A8623846F9F76AFAE5
:10884C003046FFF72CFD18B131462846FFF7E2FD04
:10885C0030682021FFF714FD00F00CF8FFF737FD0E
:10886C006A6A286A2B69811A2962204601B0BDE820
:10887C00F04018478748016821F480710160704707
:10888C00F8B5446885680E461746F9F73FFAA16BB0
:10889C0021B1F9F73FFA4FF0FF30F2BDE177616398
:1088AC00A7632663F9F736FAFFF703FD79480168E9
:1088BC0041F4007101604FF4FA612868FFF7DBFCAA
:1088CC006078A8B9616804F19000FCF797FD68B96D
:1088DC00A0634FF4FA612868FFF7D2FCFFF7F7FCAE
:1088EC00206B616B401A20631020E077606BF2BD47
:1088FC000020F2BD00BF4FF0FF30704770B500F0A4
:10890C0021F8A96B002904BFBDE87040F9F702BA41
:10891C000021A963F9F7FEF900F010F85D48016831
:10892C0021F400710160FFF7D2FC6A6B286BEB68D5
:10893C00811A29632046BDE87040184730684FF40F
:10894C00FA619DE404466568A668F9F7DFB9F0B5ED
:10895C0087B0044602A80FF25811464E1422FAF7BB
:10896C00C5FC6568A46831682068C968884740F20E
:10897C00F27720683946FFF783FC20683946FFF709
:10898C0085FC05F13C0002AA41780078C00852F839
:10899C00200008432168486300A8FFF763FC05F139
:1089AC0018000FF22011027951F822100FF2241244
:1089BC00437952F82320837935686D6811430FF29F
:1089CC001C1252F8232042EA010302680199206824
:1089DC00A847314D286840F010002860686840F0C6
:1089EC00010068602046FFF75AFC18B1686840F433
:1089FC004040686007B0F0BDF0B58468274D607BDF
:108A0C0085B040F00040009000AE207B28437060A1
:108A1C0008272046FFF743FC38B1A07B40F000400C
:108A2C00B0601027E07B2843F060FF20B85100A90C
:108A3C00134D281DFCF726FE2860B8B1617B0F2270
:108A4C00FCF7DDFE217B28681022FCF7D8FE2046BF
:108A5C00FFF725FC48B1A17B28681122FCF7CFFE5B
:108A6C00E17B28681222FCF7CAFE012005B0F0BD9C
:108A7C00163F0020D001001040420F00808D0000F6
:108A8C00703E00209B840000FF82000007830000E2
:108A9C00D1830000301000402C1000400000C0A01A
:108AAC0080B5042804BF0846FFF751FF002002BD23
:108ABC00000000000800000010000000180000007A
:108ACC00200000000000000020000000400000001A
:108ADC006000000000000000080000000000000022
:108AEC00060000000200000086000000820000006A
:108AFC00416B010060350000B80900200000000047
:108B0C00836501000200000002000000B8020000B2
:108B1C001B000000780100202C000000676501009C
:108B2C0002000000020000002375FFFF030000009C
:108B3C00EC010020040000004B6501000200000065
:108B4C00020000000175FFFF03000000F00100208F
:108B5C00080000002F650100020000000200000068
:108B6C007F0200001A000000A40100202400000075
:108B7C00136501000200000002000000B474FFFF46
:108B8C000C000000C80100201C000000F76401006C
:108B9C000200000002000000EC0100001C000000BC
:108BAC000001002044000000DB6401000200000012
:108BBC00020000009A74FFFF060000000002002073
:108BCC0004000000BF64010002000000020000006D
:108BDC007874FFFF03000000F8010020080000007B
:108BEC00A36401000200000002000000B4010000B8
:108BFC0024000000440100203400000087640100C0
:108C0C0002000000020000003474FFFF09000000A5
:108C1C00E4010020080000006B6401000200000069
:108C2C0002000000D50100006903000008020020CA
:108C3C00AE07000001207047180000000000000083
:108C4C0000000000548C0000080000000000000030
:108C5C007661722530326420252D32352E323573F3
:108C6C003D2025730D0A000000B581B016F0DAFD29
:108C7C00C046C04601B05DF804EB16F0F1BD000033
:108C8C0044F2E830C2F20000854648F67540C0F266
:108C9C0000008047FEE7000001000000000000001B
:108CAC0000000000000000000100000045B50110AC
:108CBC00BD1E000099A6011019B801106C656469FD
:108CCC0073636F6E6E656374000000004244416410
:108CDC0064726573733A25730D0A00000028000056
:108CEC00032800000129000002290000666163745A
:108CFC006F7279696E6974006C65627970617373F7
:108D0C000000000061742B6162200000636F6E66CE
:108D1C00696700007265736574000000736C6565AB
:108D2C00700000000A0B0C0D0E0F00005E235E2479
:108D3C005E2500002D412D0D0A0000002D422D0D49
:108D4C000A0000002D432D0D0A0000002D442D0DAE
:108D5C000A00000010000000500000000800000095
:108D6C008F0900004B00000064000000820000002E
:108D7C00200000000A00000004000000190F000091
:108D8C000D0A000083010001A10CD003D8070020BC
:108D9C00000143A0091420023401002004523C04B9
:108DAC001200011003103F002004041208042110CB
:108DBC0022E8082304000190082001010000083B70
:108DCC00002000015200011007C80600207807009F
:108DDC00200111C30100011003C805002008202246
:108DEC00000150026CDC02000150032C0700200330
:108DFC000D1003531E00008D04100702000000E844
:108E0C008C00000108200264F801001052EC1020C4
:108E1C0002AA090020101252182110435C041061A0
:108E2C002052AB20525420D2642052AC20525620F7
:108E3C00D27C2052AD20525820D2942052AE2052D7
:108E4C005A20D2AC2052AF20525C20D2C42052B057
:108E5C0020525E20D2DC2052B120526020D2F4206D
:108E6C0052B22052622010020405002007B0020109
:108E7C000003000114063075FFFF0600800C4AF356
:108E8C009A030001F0013C020106AF560E446155F5
:108E9C00A00A4D6F64656C204E756D62657269F049
:108EAC000302536572696119500F4669726D7761DF
:108EBC007265205265766973696F6E1CF002034807
:108ECC0061726418F00203536F667418500F4D6191
:108EDC006E756661637475726572204E616D65188E
:108EEC001003FE006578707C14046D656E74616C03
:108EFC00C9120D19F4020A100100140629006D2084
:108F0C0003CFB0F720031AB32012100852A0184B4D
:108F1C0014053012F420290952101052F030CB6C89
:108F2C000860C3B40920D28420D2B520479C085CC9
:108F3C00210C12C05C210412E804879C01746101AD
:108F4C00438D0912F0040108060020C8052043DDFA
:108F5C001E12213C2144131027B0422714216052C9
:108F6C0091401207E1100B384035002D40014002B2
:108F7C008460005D08102700F80118A384070083A3
:108F8C00057EA40306E0EA2306010088604500C3C1
:108F9C000038010304010263840000738438003537
:108FAC002C100F08047F17AC526003A302AD0163B1
:108FBC00026801FF01127C94837C06CC21016204BF
:108FCC00A111F14338381CE0020BC20110B8F301B7
:108FDC00010001A11443C5A70D52A5E0211EC00438
:108FEC0060070020C5A73961106108834002204149
:108FFC00501001010024382104F1031C2240188672
:10900C00075847B110F4B001FF002C6963411418E4
:10901C00496612783421049EE57B0312050BE5A109
:10902C0052D05C12A808210452B00452B80452C0A9
:10903C000452C80452D00452D80452E00452E8043A
:10904C0052F00452F804430008041007FCF4010029
:10905C000CF501001C04123004123C0412480412DA
:10906C005C0412700412840412900412A004140301
:10907C00010F1B0928B81A60F01203D513DC3E64EB
:10908C001104362C15F3070100011C0744617461AF
:10909C00204368617294031D7F033002737469630B
:1090AC00DCF004015374617475731AF00401436F9E
:1090BC006E66696718100A53696D706C6520424CB6
:1090CC00452050162C0270686572C7031300CC7BC8
:1090DC0012080847E823344380061010031978005F
:1090EC00002F041BD379C810062000C00200C080DA
:1090FC00FF182006051210001000020A2C3002FF87
:10910C0008808004110D1AC93440042D1F00008FF3
:10911C001FCB25A31D24051C040302E0C000308CCA
:10912C000321045238045240045248045250045251
:10913C0058045260045268045270045278045280ED
:10914C00045288041003108D00008C04173744005F
:10915C001E452C075D20036001FFFF020100011476
:02916C00020AF5
:020000040001F9
:10F00000012000F001B8000020210903263118205A
:10F01000ABBEF9E701680A680A4482604B681A448B
:10F02000C2600831016070478168C268914208D1AE
:10F0300001680A680A4482604B681A44C260083159
:10F0400001608168491C816011F8010D704738B575
:10F0500004460D46A068E168884212D120686168C4
:10F06000884208BFFFF7CCFF2068227C016802B10C
:10F070004944A16042680A44E2600830914220603D
:10F08000ECD0A068401CA06000F8015D31BD2DE906
:10F09000F0418AB000F1080105910268520801EBC5
:10F0A000C20106910021079108910168490800EB0F
:10F0B000C10108310091017901F001018DF81010B2
:10F0C00040680099400801EBC000019000200290C8
:10F0D000039006E005A8FFF79DFF0798089988426E
:10F0E00007D1059806998842F4D101980AB0BDE885
:10F0F000F08105A8FFF798FF044614F0030603D13A
:10F1000005A8FFF791FFC61C25090F2D14D105A8EE
:10F11000FFF78AFF00F10F050EE007980899884273
:10F1200004BF05A8FFF776FF0798401C079010F86A
:10F13000011D6846FFF78BFF761EEED1002DCCD067
:10F1400005A8FFF771FF0646A00800F0030003289A
:10F1500004BF05A8FFF768FFDDF800800299039F50
:10F1600006EB002008E0A8F10808A8F10801801AC1
:10F170000A6849685718394658F8082C8A1A824292
:10F18000F1D340420C18AE1CA7D0BC4206D158F8AF
:10F19000044B58F8040B2718BC42F8D00298039986
:10F1A00014F8015B884217D100980199884208BF82
:10F1B000FFF726FF009800689DF81010029009B133
:10F1C00048440290009902984968009A0144083224
:10F1D000884203910092E7D00298401C0290761E6C
:10F1E00000F8015D3FF479AFCFE7000080B501285A
:10F1F0000BD002280BD0042802D0082809D00AE03E
:10F2000000200A689047002002BD0220F9E7042090
:10F21000F7E70520F5E7FFF7F3FE00BF38B5044632
:10F22000012504E005FA00F0C0B2E1F715FDB4FADB
:10F2300084F0202800D131BD00F01CF8F2DB401F23
:10F24000C0B2E1F7B3FCF2E738B50446012504E0AB
:10F2500005FA00F0C0B2E1F71DFCB4FA84F02028F2
:10F2600000D131BD00F006F8F2DB401FC0B2E1F77B
:10F2700031FCF2E7C0F11F00C0B205FA00F14C40CA
:10F280000528704738B500793C4CA8B1E8F7C4FAB6
:10F2900005462078FF2805D12846E8F7C8FA6FF020
:10F2A000060032BD401C2070C0B2012804BF606857
:10F2B000FFF7B4FF284613E0E8F7AEFA21780A001A
:10F2C00004D1E8F7B4FA6FF0070032BD491E21708F
:10F2D000C9B229B9E8F7ABFA6068FFF7B5FF01E0FA
:10F2E000E8F7A5FA002032BD70B50446606810F05A
:10F2F0007F4F02D06FF0020070BDE8F78DFA1F4E0D
:10F300000546307828B17068FFF79EFF6068FFF708
:10F3100085FF606870602846E8F789FA002070BDB4
:10F3200080B5406810F07F4F00D00DE0FFF776FF0A
:10F33000002002BD80B5406810F07F4F00D003E090
:10F34000FFF782FF002002BD6FF0020002BD1CB576
:10F350000446A168606808601420E8F700FC01908A
:10F3600010B96FF0030016BD002000900F21A368B4
:10F370000198034AE1F705FC002016BD2009002092
:10F38000EDF1010010B50446E1F770FB00B101207A
:10F390002071002010BD80B5E1F768FD002002BD9E
:10F3A00010B50446E1F75BFB6060002010BD10B5AE
:10F3B00004466068E1F758FBA060002010BD000023
:10F3C0004275696C6456657273696F6E0000000067
:10F3D00042445F4144445200303030343365323669
:10F3E00030306132000000004465766963654E612B
:10F3F0006D650000426C655F50657269706865728A
:10F40000616C00005561727442617564726174656B
:10F410000000000031313532303000005561727427
:10F420004461746142697473000000003800000098
:10F430005561727453746F704269747300000000F8
:10F4400031000000486F737444656570536C6565E6
:10F4500070456E0030000000486F73744576656E2D
:10F4600074730000426441646472456E620000007F
:10F47000416476496E744D696E00000033320000BD
:10F48000416476496E744D61780000005363616E8B
:10F49000496E74005363616E57696E646F77000044
:10F4A00031380000436F6E6E656374496E744D6948
:10F4B0006E00000031360000436F6E6E6563744964
:10F4C0006E744D617800000053657276696365550E
:10F4D0005549440046303030433045312D303435C5
:10F4E000312D343030302D423030302D303030300E
:10F4F0003030303030303030000000002D436F6D40
:10F500006D616E644D6F64652D000000526573651A
:10F510007450656E64696E6700000000446973632F
:10F520006F7665727950656E64696E6700000000E1
:10F53000436F6E6669674F6B00000000436F6E6635
:10F5400069674572726F72002D424C452D436F6E94
:10F550006E656374696F6E55700000002D424C45F6
:10F560002D436F6E6E656374696F6E446F776E00C6
:10F570002D424C452D4279706173734D6F64652D3A
:10F58000000000002D536C6565704D6F64652D00A3
:10F59000436F6E6E65637454696D656F75740000BA
:10F5A0004164764F6B0000007B756E6B6E6F776EFB
:10F5B0002D696E7374616E63652D6E616D657D007E
:10F5C0007B656D7074792D696E7374616E63652DE2
:10F5D0006E616D657D0000007B7374617469632DDD
:10F5E000696E7374616E63652D6E616D657D00007B
:10F5F0008F3F00008F3F01008F3F02008F3F0300CD
:10F60000903F00018F3F0101903F0002903F0003B7
:10F610008F3F01048F3F00058F1208048F3F0004C5
:10F620008F3F0006513F00007F3F01003F3F040035
:10F630003F3F02003F3F01007F3F020019E050F8CA
:10F64000041BCB0744BFA9F101035918121F002363
:10F65000042A41F8043BF9D25FEA827C0B4604D5C8
:10F660004FF0000CA1F800C09B1CD10744BF002143
:10F67000197050F8042B002AE1D17047DFF800F030
:10F6800055C0011080B50B48E5F758FF0420E1F79D
:10F69000E3FA0820E1F7E0FAE8F7B6F9E8F7D2F97B
:10F6A000E6F7B6FBE7F756FAE4F74AFBFFF7E6FFA3
:10F6B000002002BDF008002053797374656D20436B
:10F6C0006F6E66696775726174696F6E20536574D9
:10F6D00074696E6773202D2056657273696F6E2092
:10F6E000312E300D0A000000188D0000456F00001B
:10F6F000208D00007F700000F88C0000FB6F000080
:10F70000C88C000077700000288D00009170000008
:10F71000048D0000A37000007FC80110C9BC011057
:10F7200051B2011037C20110BDAD0110C1B10110BD
:10F73000E909000071BA011069BB011021C0011074
:10F74000EBC70CEEC910F1CB14F4CE14F74F21FA2D
:10F750005429FD5C35006C56011F6A02299C00008B
:10F7600040F701000A0700000010004015000000EB
:10F77000060000000201FFFFB8F70100383A002040
:10F7800068F7010000000000000000000000000019
:10F7900000000000000000B000405104E0C000F094
:10F7A00000000000000000B000405104E1C000F083
:10F7B0001000000090F70100E78600005587000068
:10F7C0007F8500008F8500008D8800000189000082
:10F7D0000989000077870000238800002588000041
:10F7E00010B5074979441831064C7C44163404E0BE
:10F7F0000A68081D114488470146A142F8D110BD8E
:10F80000FC92FEFF3C94FEFFFFFFFFFF600900201B
:10F8100004000000000000000000000014000000D0
:10F82000448C000018000000DFF800F059C50110FA
:10F830000548012808BFE2F7F4BA704703480128D9
:10F8400008BFFFF7F1BF7047010000000100000092
:10F850000A18232A242A252A262A272A282A292A56
:10F860002A2A502A0200000050F80100E9F7E8F9BE
:10F87000002803D0FFF7B4FFFFF7E0FF0020FFF7F9
:06F8800001FFE2F76DFA42
:10FFA80000008006100082FFFDFF58003AFFBFF3F3
:10FFB800FFFFFFFFFFFFFFFFFFFFFFFFFFFFFFFF49
:10FFC800FFFFFFFFFFFFFFFFFFFFFFFFFFFFFFFF39
:10FFD800C505FEC5FFFFFFFFC5FFFFFFC5C5C5FF80
:10FFE800C5C5C5FF00000000FFFFFFFFFFFFFFFFC3
:08FFF800FFFFFFFFFFFFFFFF09
:0400000500008C8DDE
:00000001FF
